:020000040000FA
:200000000C9449020C9466020C94B12A0C9466020C940F310C9466020C9466020C946F0269
:200020000C9466020C9466020C9466020C9466020C9466020C94D6330C9466020C946602DF
:200040000C9466020C9466020C9466020C9466020C9466020C9466020C94692F0C94660230
:200060000C946602760AAD09FA09AF0AAF0AA40AA40AA40A520AFA09C4098C0A3F0A3F0A6F
:20008000FE092A0A170A3F0A3F0A3F0A3F0AFA09FA09670AA40A860AF509A40AA40AA40A23
:2000A000A40AA40AA40A740A990EB30ED80ED80EE30FE30FE30FC90FD60EE30FE30FE30F1C
:2000C000E30FE30FD90FE30FE30FE30FE30FE30FE30FE30FE30FE30FE30FE30FE30FE30F0A
:2000E000E30FE30FE30FE30FE30FE30FE30FE30F4E0E520EE30F520E520E590EE30FE30FB7
:20010000540E540E5F0E790EE30FB80FE30FE30E4A0F004E4554574F524B004A4F494E00D8
:200120004C45415645004D41494C00494E424F5800434F4D504F534500415544494F0050D7
:200140004C4159005245434F52440053454E534F52530054454D500054494D4500434C4F8A
:20016000434B0053595354454D00434F4E464947004C434400434F4E54525354005343526E
:200180004F4C4C494E47004E414D4500554E4954530054454D5000524144494F0050414E62
:2001A000204944004348414E4E454C00434C4F434B00434F4E4E45435400444542554700BC
:2001C000545854505245560053544F524147450046494C455300464F524D415400465700F4
:2001E00055504752414445005245424F4F5400A502FC01EF01EF011201F31903EF01230271
:20020000FC010902130100000016021602FC0109021B01531A0309020902FC0116022001B2
:200220001F1A02FC014A022302300226010000003D023D02230230022B01901803300230AE
:200240000223023D0231010E1902230271024A0257023901000000640264024A0257023FB6
:20026000018C1903570257024A02640244019618024A028B0271027E024B010000007E02E4
:200280007E0271027E0253019518037102A5028B0298025801000000980298028B029802F2
:2002A0005D01981A038B02EF01A502B2026301000000A9036803A502BF026A010000015BA9
:2002C00003E602B202CC027101000001D902D902BF02CC027501911803CC02CC02BF02D9A1
:2002E000027D01451B02BF02F302B202E6028701921802E6020D03B20200038C010000005A
:2003000000030003F30200039201931803F3023403B2021A039701000000270327030D03A5
:200320001A039D019418031A031A030D032703A401F31A020D034103B2023403AC01BA1A6B
:200340000234034E03B2024103B201FB180241035B03B2024E03BA01D418024E03BF02B23F
:20036000025B03C001C11802B2028F03A5027503C8010000008203820368037503D0011580
:2003800019037503750368038203D6017319026803A903A5029C03DD010000009C039C0383
:2003A0008F039C03E0018E18038F03B202A502A903E8018F1802090008010900080109002A
:2003C000080109000801090008010A0010020A0010020B0020040000000000000000000089
:2003E00000000000000000000000722E3028000010080000400285918080941994989188A3
:2004000015981599848095999598000000004004000002024420A5199589A4B80511A4B0D4
:2004200015191501059991892020809151050111C3818385859195098595950D159824205A
:20044000819141038187420642204412051102048490030000103F065B4F666D7D077F6FC7
:20046000777C395E7971004053332944494E2EE351D1635262E2CDC34FCFD2ADEDF2A8A3BB
:20048000B260E061E19283888DC80444D050E884C40011241FBECFEFD8E0DEBFCDBF13E0FA
:2004A000A0E0B1E0E0E8FDE602C005900D92A430B107D9F717E0A4E0B3E001C01D92A03CD4
:2004C000B107E1F70E944C050C94BE360C9400008FEF9FEF089508958091250708951F9294
:2004E0000F920FB60F9211242F933F934F938F939F93AF93BF93EF93FF938091000190911B
:20050000010101979093010180930001019609F048C184E090E090930101809300012091B1
:20052000200730912107203131050CF048C080912207882309F080C0F901E050F94F80818F
:2005400090E09093890080938800C90101969093210780932007409709F023C181E08093D6
:2005600022073091BA07332331F48091B9078F5F8093B90716C120916807E22FF0E0EE0FEE
:20058000FF1FEE0FFF1FDF01A759B84F80E597E08D939C93E559F84F11821082233119F405
:2005A0001092680703C02F5F2093680731503093BA07809167078F5F80936707F2C0809101
:2005C00023078823C9F5F901E050F94F808190E09093890080938800C901019690932107B2
:2005E00080932007809709F0DCC081E0809323073091BA07332309F471C020916807E22F40
:20060000F0E0EE0FFF1FEE0FFF1FDF01A759B84F80E597E08D939C93E559F84F1182108218
:20062000233119F41092680703C02F5F2093680731503093BA0776C080912707909128070B
:200640002817390709F0ADC08FEF9FEF909328078093270780912407882309F46DC0409134
:20066000BA0720313105ACF581E080932207442331F48091B9078F5F8093B90723C0209142
:200680006807E22FF0E0EE0FFF1FEE0FFF1FDF01A759B84F80E597E08D939C93E559F84F3D
:2006A00011821082233119F41092680703C02F5F2093680741504093BA07809167078F5F9E
:2006C0008093670780E190E0909321078093200768C081E080932307442331F48091B90720
:2006E0008F5F8093B90723C020916807E22FF0E0EE0FFF1FEE0FFF1FDF01A759B84F80E5D3
:2007000097E08D939C93E559F84F11821082233119F41092680703C02F5F209368074150F3
:200720004093BA07809167078F5F80936707109221071092200735C081E08093260730914D
:20074000BA07332331F48091B9078F5F8093B90723C020916807E22FF0E0EE0FFF1FEE0FCF
:20076000FF1FDF01A759B84F80E597E08D939C93E559F84F11821082233119F4109268072D
:2007800003C02F5F2093680731503093BA07809167078F5F80936707809181008E7F809341
:2007A0008100FF91EF91BF91AF919F918F914F913F912F910F900FBE0F901F9018958091E0
:2007C00004038823C1F0809125078823A1F010922507809181008E7F8093810081ED0E942C
:2007E000E52B8091290790912A070E943D2510922A071092290708951F93CF93DF93EC019D
:20080000162F809104038823F1F180912507882311F00E94DF0361E0CE010E94002290938A
:200820002A0780932907892B71F1109324071092220721E020932307109221071092200724
:200840008FEF9FEF90932807809327072093250710922607E0E0F7E08FE7819397E0E031A2
:20086000F907D9F78091810081608093810081ED0E94CB2B60E070E080E597E00E948B31D1
:2008800020E030E002C02FEF3FEFC901DF91CF911F91089580910403882309F459C0809169
:2008A0002507882309F454C080912207882309F12091290730912A0740E150E060E070E0BD
:2008C00080E097E00E94921C603171058105910570F4709328076093270780912407882330
:2008E00041F08091290790912A070E94E81B1092220780912307882319F120912907309132
:200900002A0740E150E060E070E080E197E00E94921C603171058105910580F4CB01409664
:20092000909328078093270780912407882341F08091290790912A070E94E81B1092230708
:2009400080912607882321F00E94DF031092260708950E945B310E945331E4E6F0E08081BE
:2009600088608083779A089580910403882311F00E94A9046F9A77980E9454310E944C316D
:2009800010922A0710922907109225071092260780916400877F809364008FEF90E0909312
:2009A000870080938600109285001092840087E086BB82E080936F0082E88093800088E1D8
:2009C0008093810081E08093040380E090E00895A89580916000887F806180936000A89555
:2009E00080916000886180936000FFCF0F931F93DF93CF930F92CDB7DEB78C01CB0161E0E0
:200A00000E949730C8010E9462308FB78983F894789483EE0E94CB2B83E00E94CC3080E418
:200A20009DE0A3E0B0E020E031EE45EF55E0629917C00097A105B10521F00197A109B109CC
:200A400013C081E00E94CC300E94572B629BFECF89818FBF0F90CF91DF911F910F91089522
:200A600080E49DE0A3E0B0E0211531054105510529F02150304040405040D9CFA89580917A
:200A80006000887F806180936000A89580916000886180936000FFCF0F931F93DF93CF939B
:200AA000CDB7DEB728970FB6F894DEBF0FBECDBF8091FEDF9091FFDF9B838A838FEF80936E
:200AC0007E0083E080937F008FE18093640080B7806880BF8FB78983F89480E880936100A4
:200AE00081E08093610089818FBF84E083BF0E946531882309F4FFCF25E033E042E060E2F9
:200B000070E089E293E00E94003221E133E042E060E470E089E693E00E9400322DE133E031
:200B200042E060E870E089EE93E00E9400320E94EF06882309F4FFCF0E946E34892B09F03F
:200B4000FFCF0E94A634892B09F0FFCF0E94932A892B09F0FFCF0E940631892B09F0FFCFA2
:200B6000FE01349685E0DF011D928A95E9F74C8140644C835D81506C5D836E8167606E8358
:200B800083EF8F8382E0888773EF0E94902C892B09F0FFCF83EE0E94CB2B82E091E00E94A7
:200BA000623080E00E94CC3088E893E124E630E0F9013197F1F70197D9F781E50E94CB2B97
:200BC00088E893E124E630E0F9013197F1F70197D9F781ED0E94CB2B88E893E124E630E001
:200BE000F9013197F1F70197D9F783E60E94CB2B88E893E124E630E0F9013197F1F70197A2
:200C0000D9F782E50E94CB2B20E137E204E610E005C0C8010197F1F72150304021153105B6
:200C2000C1F783EE0E94E52B88E893E1F8013197F1F70197D9F783EE0E94CB2B88EE93E0F2
:200C4000F8013197F1F70197D9F781E00E94CC3080E197E2F8013197F1F70197D9F780E039
:200C60000E94CC3020E137E2D4CFCF93DF9327E040E460E08EE10E94921B88EC8A95F1F7A1
:200C80000E94B61B80E00E94C91BEC018FEFCF3FD807C1F30E94A71B9E01442737FD409578
:200CA000542F60E070E381E190E00E948736C901DF91CF91089564E070E086E10E94472CA6
:200CC000089564E070E086E10E94472C82E90E94CB2B80E090E00895FF920F931F939C0175
:200CE00068EE73E00E943E36082FF92EC90168EE73E00E943E36FB0124E0EE0FFF1F2A9574
:200D0000E1F7802F9F2D64E670E00E943E36482F192F802F9F2D64E670E00E943E369B014A
:200D20002E0F3F1F94E0220F331F9A95E1F7842F912F6AE070E00E943E36260F371F84E008
:200D4000220F331F8A95E1F7842F912F6AE070E00E943E36282B392BC9011F910F91FF9096
:200D60000895FC01EF70F070AC01452F552742954F7028EE33E0429FB001439F700D529FDC
:200D8000700D11246E0F7F1F9C01207F3070A4E036952795AA95E1F7A901F3E0440F551F44
:200DA000FA95E1F7220F331F420F531F640F751F80709F70892F992724E630E0AC01429F60
:200DC000C001439F900D529F900D1124680F791FCB0108951092E9040E94443308954EEF16
:200DE00056E06AEE74E086E40E940C33882319F081E08093E9048091E9040895FC01808118
:200E0000853189F0863128F48131F9F08131B8F007C0873171F0873148F0883181F40CC011
:200E20008AE19CE014C084E49DE011C088E79BE00EC08DE59CE00BC086E09DE008C0809114
:200E4000C10080688093C100089585E29EE0BF010E948B31882329F48091C10080688093E0
:200E6000C10008959C0180914C07882319F02FEF3FEF04C0C9010E94A4279C01C901089514
:200E800021E040E06CE080E10E946E27249A2C9A80E090E008950E945C2A80E090E00895C7
:200EA0000E944A040895FC0180810E948A2B0895DF93CF9300D00F92CDB7DEB7609133072A
:200EC000CE0101960E947B15898124E68202C00111242A81332727FD309560E0820F931F7B
:200EE0000E9497308091300590E021E030E08227932780933005882321F084EC0E94CB2B53
:200F000003C084EC0E94E52B0F900F900F90CF91DF910895CF93DF930E943506EC0163E0C1
:200F200070E087E10E94472C87E0C13DD8078CF083E80E94CB2B89E0C53CD80754F088E824
:200F40000E94CB2B8AE0C13FD8071CF08DE80E94CB2B80914C07882359F4C852DA4044F4CF
:200F600081E080934C0782EE0E94CB2B0E94E51BDF91CF9108950E94102E08950E94292F1C
:200F800008950E94C12E089580914F01882339F00E94BB2A8093310510924F0108950E9450
:200FA000BB2A982F80913105981741F09093310561E375E08FED97E00E948B310895BF922D
:200FC000CF92DF92EF92FF920F931F93DF93CF93CDB7DEB768970FB6F894DEBF0FBECDBFA6
:200FE000FC01B08089E792E00E9462187C0182E0898384E0B81609F451C18B1540F0A1E049
:20100000BA1671F0B2E0BB1609F0A9C299C0E8E0BE1609F46BC1F0E1BF1609F0A0C28CC16C
:2010200080914F078A3199F18B31C8F4843109F453C0853150F48D3009F44CC08E3009F44C
:2010400064C08A3009F08BC21DC0883109F45BC0893108F05AC0853109F081C23BC08E3146
:2010600091F18F3128F48C3101F18D3128F516C0843209F454C08B3209F4B7C1813209F00D
:201080006EC245C089E792E00E94381848C187E091E00E94E82FB0923A0769C287E091E027
:2010A0000E94E82FB092340762C28EE091E00E94E82FB09235075BC28EE091E00E94E82F0B
:2010C000B092370754C28EE091E00E94E82FB09236074DC280E026C180E00E94FF0F61E0BC
:2010E0000E9497300E94282B2C8B3D8B4E8B5F8B688FDE011296FE01749685E001900D9234
:201100008150E1F788C080E091C080E00FC18E01095F1F4F46E050E063E171E007C08E0157
:20112000095F1F4F44E050E06FE171E0C8010E94F23580914C07882309F0ABC041E08DC071
:2011400080914F078A3199F18B31C8F4843109F44CC0853150F48D3009F445C08E3009F439
:201160006BC08A3009F0FBC11DC0883109F45DC0893108F061C0853109F0F1C134C08E313E
:2011800059F18F3128F48C3139F18D31F0F416C0843209F466C08B3209F427C1813209F0A3
:2011A000DEC14CC089E792E00E944118B8C083E291E00E94E82F10923A07D9C183E291E04D
:2011C0000E94E82F10923407D2C183E391E00E94E82F10923707CBC18BE291E00E94E82F53
:2011E00010923607C4C181E09DC081E00E94FF0F61E00E9497300E94282B2C8B3D8B4E8BC5
:201200005F8B688FDE011296FE01749685E001900D928150E1F70E94F10F8E834A815B81C5
:201220006C817D810E94F42AA2C181E00E94FF0F61E00E9497309BC181E078C08E01095FF9
:201240001F4F46E050E063E171E0C8010E94F23580914C078823E9F440E064E375E0C80132
:2012600011C044E050E06FE171E0CE0107960E94F23580914C07882361F440E064E375E053
:20128000CE0107960E94FA1D84E395E00E9462306EC189E191E00E94E82F69C180914F07C5
:2012A000853101F1863140F48D30E1F08E30E1F08A3009F054C109C0813261F08B3209F42F
:2012C00094C0893109F04BC10FC089E792E00E944C1825C00E946C02882309F486C00E94BF
:2012E000DF0383C082E01EC082E020C080914F078E30D9F08F3030F48A3069F08D3009F0AD
:201300002EC10FC0893189F08B3209F46EC0853109F025C106C089E792E00E945718BC01E9
:201320001FC183E00E944E1622C183E00E94FF0F60E00E94002E1BC180914F0790E0FC01AE
:201340003A97E232F10508F0FFC0EE5CFF4FEE0FFF1F0590F491E02D0994C7010E9486187C
:201360000E94E82F81E00E94CC300E94572B83E08983D7011A96ED91FC911B973097D1F154
:20138000CE010196099536C00E94F10F80933D070E94F80F0E94282B2C8B3D8B4E8B5F8B7A
:2013A000688FDE011296FE01749685E001900D928150E1F780913D078E834A815B816C816E
:2013C0007D810E94F42A5BE2C52E57E0D52E88E290E0F60161916F018C010F5F1F4F0E94A7
:2013E0008A35C80109341105A1F7C7010E9486180E94E82F8AE080934F07B9C00E94F10FCB
:20140000809331070E94F80F4BE2C42E47E0D42E88E290E0D6016D916D018C010F5F1F4F0A
:201420000E948A35C80109341105A1F7DECF3BE2C32E37E0D32E88E290E0F60161916F0191
:201440008C010F5F1F4F0E948A35C80109341105A1F7CBCF0E94F80F2BE2C22E27E0D22EC7
:2014600088E290E0D6016D916D018C010F5F1F4F0E948A35C80109341105A1F7B6CF9BE2CF
:20148000C92E97E0D92E88E290E0F60161916F018C010F5F1F4F0E948A35C80109341105BE
:2014A000A1F7A3CFC7010E9486180E94E82F83E08983D7011A96ED91FC911B97309719F0DD
:2014C000CE010196099581E00E94CC3093CF0E946C02882331F460E084E395E00E94FC030A
:2014E00046C00E94DF0343C085E285CFC7010E9486180E94E82FD7011A96ED91FC911B979E
:201500003097A9F1CE010196099531C00E946B0283E60E94E52B6ECF84E00E944E160E9402
:201520003B168BE2C82E87E0D82E88E290E0F60161916F018C010F5F1F4F0E948A35C801C4
:2015400009341105A1F751CF8AE391E00E94E82F83E00E94CC300E94572B8BE04CCFB70186
:201560006E157F0521F04981C7010E949718B0923305BB2019F180913205882341F58091D7
:201580005101882339F0109251012CE231E040E050E00BC0809150010E94AA3481E08093A1
:2015A000320520E530E040E050E063E375E08FED97E00E9400358093500109C0809150019B
:2015C0000E94AA3481E0809351011092320568960FB6F894DEBF0FBECDBFCF91DF911F9127
:2015E0000F91FF90EF90DF90CF90BF900895EF92FF920F931F93DF93CF930F92CDB7DEB78F
:2016000080914F07882309F06BC083E08983BE016F5F7F4F81E00E944F3383EE0E94CB2B3C
:2016200082ED0E94E52B8DEA0E94E52B64E070E082E10E94472C65E070E081E10E94002C8F
:201640008FEF9FEF90934E0780934D0781E00E94CC3083E491E00E94E82F87E290E00E9494
:201660007535E82EFF2400E010E0102F0F2DFE2CEE2486E290E00E94753590E0A0E0B0E05C
:20168000E82AF92A0A2B1B2B102F0F2DFE2CEE2485E290E00E94753590E0A0E0B0E0E82A2E
:2016A000F92A0A2B1B2B102F0F2DFE2CEE2484E290E00E94753590E0A0E0B0E0E82AF92AFE
:2016C0000A2B1B2B8DE0E81680EFF8068EEB08078AEB180711F48CE301C08BE380934F078F
:2016E0000F90CF91DF911F910F91FF90EF900895EF92FF921F93CF93DF93EC0185E0E82E80
:20170000F12CEC0EFD1EF70111818DEA0E94E52B82ED0E94CB2B64E070E082E10E94472CD1
:2017200064E070E081E10E94002C89818C3D18F481E60E94E52B8981883C18F480EE0E9403
:20174000E52B8981863918F480E60E94E52B123109F44EC01331A0F4153071F1163040F445
:201760001330F1F0143020F5123009F051C01CC01F3051F11131C1F1163009F049C020C017
:201780001A31F1F11B3138F4143151F1143120F11931F1F51DC01E31B8F1103FC9F52CC0C9
:2017A000CE010E948E1440C0CE010E9460133CC0CE010E946F1138C0CE010E945E1434C076
:2017C000CE010E94CA1130C0CE010E9450112CC0CE010E945F1228C0CE010E944C1124C093
:2017E000CE010E944D1120C0CE010E944E111CC0CE010E944F1118C0CE010E94AC1214C0E2
:20180000CE010E940B1210C0CE010E9439120CC08091C10080688093C1006A817B81F70175
:2018200040818CE10E945111DF91CF911F91FF90EF900895DF93CF930F92CDB7DEB78091AC
:20184000C10080688093C10080914F078430A1F0853028F4813001F1833009F510C08930B1
:2018600019F08732E1F415C082ED0E94E52B8DEA0E94E52B8AE01BC082E591E012C08BE058
:201880008983BE016F5F7F4F81E00E944F3384E00EC083E691E005C080E791E002C087E783
:2018A00091E00E94E82F83E00E94CC308BE080934F070F90CF91DF910895EF92FF920F9369
:2018C0001F93DF93CF930F92CDB7DEB78091C10080688093C10080914F078B3331F08C3335
:2018E00091F0833309F08AC02BC084E08983BE016F5F7F4F81E00E944F338DE791E00E94AC
:20190000E82F8DE379C083E00E94CC3085E991E00E94E82F83E08983BE016F5F7F4F81E043
:201920000E944F3380E090EBA6E1B0E08093540790935507A0935607B093570783E35CC0F1
:2019400088EA0E94E52B83EA0E94E52B82ED0E94E52B8DEA0E94E52B64E070E082E10E9461
:20196000472C65E070E081E10E94002C87E290E00E948D327C01909342058093410500971E
:20198000E9F1109250071092510710925207109253078C01095F1F4F609154077091550777
:2019A000809156079091570720E230E040E050E00E94642986E0F701808380E290E096835D
:2019C00085831182128213821482B70187E20E944F338091500790915107A0915207B091BC
:2019E00053072AE0B695A795979587952A95D1F761E00E94973084E380934F070F90CF91B4
:201A0000DF911F910F91FF90EF900895DF93CF9300D0CDB7DEB78091C10080688093C10010
:201A200080914F078D3319F08E3349F512C08FE0898382E08A83BE016F5F7F4F84E00E945A
:201A40004F3386EB91E00E94E82F86E380934F0716C06DE084E290E00E948A3560EF85E287
:201A600090E00E948A356DEA86E290E00E948A356AEB87E290E00E948A350E94E8040F9049
:201A80000F90CF91DF910895EF92FF920F931F93DF93CF9300D000D0CDB7DEB78C0189E74A
:201AA00092E00E9462189C0180914F07873031F0863319F1853009F0BDC007C060E0F801CE
:201AC000828193810E94002E0FC0F8018281938190934E0780934D0743E0B901C9010E9418
:201AE000971881E00E94CC308AE080934F078091C10080688093C1009DC0F801938180E00D
:201B0000228130E0822B932B9093590780935807958180E0248130E0822B932B90935B0797
:201B200080935A078091C10080688093C10087E290E00E947535E82EFF2400E010E0102F36
:201B40000F2DFE2CEE2486E290E00E94753590E0A0E0B0E0E82AF92A0A2B1B2B102F0F2D3E
:201B6000FE2CEE2485E290E00E94753590E0A0E0B0E0E82AF92A0A2B1B2B102F0F2DFE2C31
:201B8000EE2484E290E00E94753590E0A0E0B0E0E82AF92A0A2B1B2BFEEBEF16FAEBFF0609
:201BA000FEEF0F07FAEC1F07D1F489E08983809131078A8380912F07909130079C838B83BA
:201BC000BE016F5F7F4F84E00E944F338DEC91E00E94E82F84E00E94CC308FE229C089E7B3
:201BE00092E00E94321843E0BC010E949718809137078823E1F089E08983809131078A83C0
:201C000080912F07909130079C838B83BE016F5F7F4F84E00E944F338DEC91E00E94E82F72
:201C200084E00E94CC300E94572B81E001C08AE080934F070F900F900F900F90CF91DF913D
:201C40001F910F91FF90EF900895AF92BF92CF92DF92EF92FF920F931F93DF93CF9300D01B
:201C60000F92CDB7DEB789E792E00E9462188C018091C10080688093C10080914F0790E0BA
:201C8000FC013197E533F10508F09DC1EC5AFF4FEE0FFF1F0590F491E02D09948DED91E0BD
:201CA0000E94E82F87E28DC187EE91E00E94E82F3EC083E00E94CC308CEE91E05EC188EA9A
:201CC0000E94CB2B83EA0E94CB2B64E070E082E10E94472C64E070E081E10E94002C8BE02C
:201CE0008983BE016F5F7F4F81E00E944F3380E368C187EF91E00E94E82F40E060E070E01C
:201D000089E20E9451116DE084E290E00E948A3560EF85E290E00E948A356EEF86E290E014
:201D20000E948A356AEC87E290E00E948A358BE048C188EA0E94CB2B83EA0E94CB2B64E0EB
:201D400070E082E10E94472C64E070E081E10E94002C8BE08983BE016F5F7F4F81E00E9422
:201D60004F3383E02EC188EA0E94E52B83EA0E94E52B82ED0E94E52B8DEA0E94E52B64E0BE
:201D800070E082E10E94472C65E070E081E10E94002CC8010E9486180E94E82F0E94572BD0
:201DA0008FEF9FEF90934E0780934D078AE009C18FE08A831B82BE016E5F7F4F82E00E948D
:201DC0004F3385E0FEC0E0904105F0904205A0905007B0905107C0905207D09053078701D7
:201DE000095F1F4F609154077091550780915607909157076A0D7B1D8C1D9D1D20E230E0F3
:201E000040E050E00E94642986E0F701808380E290E096838583A182B282C382D482B70145
:201E200087E20E944F338091500790915107A0915207B0915307FAE0B695A7959795879566
:201E4000FA95D1F761E00E9497308091500790915107A0915207B09153078096A11DB11DD9
:201E60008093500790935107A0935207B09353078050904EA140B04009F0A5C08091410520
:201E8000909142050E94CD3287EE91E00E94E82F85E397C084E08983BE016F5F7F4F81E0AF
:201EA0000E944F3387E290E00E947535E82EFF2400E010E0102F0F2DFE2CEE2486E290E041
:201EC0000E94753590E0A0E0B0E0E82AF92A0A2B1B2B102F0F2DFE2CEE2485E290E00E9456
:201EE000753590E0A0E0B0E0E82AF92A0A2B1B2B102F0F2DFE2CEE2484E290E00E9475352F
:201F000090E0A0E0B0E0E82AF92A0A2B1B2B2DE0E21620EFF2062EEB02072AEB120789F4B8
:201F20006EEB84E290E00E948A356AEB85E290E00E948A356EEF86E290E00E948A356AEC98
:201F400010C06DE084E290E00E948A3560EF85E290E00E948A356DEA86E290E00E948A3516
:201F60006AEB87E290E00E948A350E94E8042BC083E00E94CC3080E092E00E94E82F83E06A
:201F80008983BE016F5F7F4F81E00E944F3383E318C082ED0E94E52B8DEA0E94CB2B8BE07C
:201FA0008983BE016F5F7F4F81E00E944F3389E008C08AE092E00E94E82F84E00E94CC306D
:201FC00080E180934F070F900F900F90CF91DF911F910F91FF90EF90DF90CF90BF90AF90D0
:201FE0000895E0914305F09144058081918108951092470560E080E00E94D72D089590911F
:202000004805992321F0913009F0D6C09FC0823009F45DC0833030F4882341F0813009F0CE
:20202000CBC02EC0833009F0C7C070C0E0914305F0914405408151812091450530914605A7
:20204000CA01822393238217930729F4809590958423952308C088279927821B930B82235A
:202060009323840F951F91838083208131818091490590914A05821793070CF47DC098C062
:20208000E0914305F0914405208131814091450550914605C90184239523892B19F4242BEA
:2020A000352B08C088279927841B950B84239523281B390B318320832081318180914B0559
:2020C00090914C05281739070CF46CC071C0809145059091460534E0880F991F3A95E1F7E1
:2020E0009093460580934505892B31F480E090EF909346058093450580914705880F80938B
:202100004705803109F058C080E81DC0809145059091460524E0969587952A95E1F79093A0
:20212000460580934505892B31F48FE090E09093460580934505809147058695809347059D
:202140008823D1F581E08093470536C0882319F0813091F516C0E0914305F0914405808113
:2021600091812091490530914A05019691838083019782179307E0F080914B0590914C0522
:2021800015C0E0914305F09144058081918120914B0530914C05019791838083019628173C
:2021A000390730F08091490590914A059183808360914705609502C060914705809147054B
:2021C0000E94D72DE0914305F0914405808191810895EF92FF920F931F93DF93CF93CDB768
:2021E000DEB72B970FB6F894DEBF0FBECDBFE982FA820B831C832D833E83E42F4F835887F8
:202200006987972F7A878B872B813C8149815A8168857985F92F8D819E8190934A05809322
:20222000490530934C0520934B05EE2319F089E090E002C08FE090E09093460580934505DA
:202240005093440540934305E093480521E030E081E004C0880F81602F5F3F4F2617370732
:20226000C8F390E002C0880F991FFA95E2F780934705682F60950E94D72D80E090E02B9698
:202280000FB6F894DEBF0FBECDBFCF91DF911F910F91FF90EF9008950895089508950895B8
:2022A0000895DF93CF9300D000D000D0CDB7DEB7FE0131969DE099837283618392E0938364
:2022C0004D838E83BF0186E00E944F3326960FB6F894DEBF0FBECDBFCF91DF910895FC0166
:2022E0006281738145818091C10080688093C10080914F07873239F48AE10E9451118DE288
:2023000080934F0708958BE10E9451110895AF92BF92CF92DF92EF92FF920F931F93CF937E
:20232000DF93B82EA92E7B01D42E122FC32E022F0B5F802F90E00E948D32EC01009719F412
:202340002FEF3FEF1BC08DE08883FA82E9821F5F1B831150DC829E012B5F3F4F412F5C2D6C
:202360006B2D7A2DC9010E940136BE01802F0E944F33CE010E94CD3220E030E0C901DF912F
:20238000CF911F910F91FF90EF90DF90CF90BF90AF900895CF92DF92EF92FF920F931F934E
:2023A000CF93DF938C01FC01C280D380E580F7808F2D90E00E948D32292FC82FD92F2097B3
:2023C00059F48091C10080688093C1004E2DB6018BE10E94511116C0C80108964F2D50E097
:2023E000BC018C2F922F0E9401368091C10080688093C1004E2DB6018AE10E945111CE01CD
:202400000E94CD32DF91CF911F910F91FF90EF90DF90CF900895CF93DF93FC01C281D3811A
:2024200095818091C10080688093C10080914F078031E1F480916007981751F082E192E0CE
:202440000E94E82F60E0CE010E94002E83E009C081E292E00E94E82F60E0CE010E94002E4B
:2024600084E00E94CC308BE080934F07DF91CF9108958091C10080688093C10090914F0714
:20248000892F8B518330D0F49A3019F09031B1F40BC086E292E00E94E82F83E00E94CC3099
:2024A0008BE080934F07089580E392E00E94E82F83E00E94CC308BE080934F070895DF923A
:2024C000EF92FF920F931F93DF93CF93CDB7DEB72C970FB6F894DEBF0FBECDBFFC01E28040
:2024E000F380D5808091C10080688093C1008E010F5F1F4F85E289838EE397E0FC01019032
:202500000020E9F7EF53F740D8011196EC93BC01CE0103960E940A36F801218130E02E5F04
:202520003F4F4D2DB701C8010E9487118F5F9F4F29F44D2DB7018BE10E9451112C960FB6B6
:20254000F894DEBF0FBECDBFCF91DF911F910F91FF90EF90DF900895BF92CF92DF92EF921B
:20256000FF920F931F93DF93CF93CDB7DEB728970FB6F894DEBF0FBECDBFFC01C280D380F1
:20258000B5808091C10080688093C10080914C07882339F489E090E00E948D327C010097EE
:2025A00031F44B2DB6018BE10E94511179C08E010F5F1F4F22E030E040E050E06EEF7FE293
:2025C00089E190E00E9464298E010D5F1F4F22E030E040E050E06EEF7FE888E190E00E94E8
:2025E00064298E010B5F1F4F22E030E040E050E06EEF7FE389E190E00E9464298E01095FC6
:202600001F4F22E030E040E050E06EEF7FEA88E190E00E94642981EFF701808381E081834C
:2026200089E0828380E092E09483838380915C0790915D0796838583809158079091590732
:202640009087878380915E0790915F079287818780915A0790915B079487838789819A81FC
:20266000968785878B819C81908B87878D819E81928B818B8F819885948B838B25E130E019
:202680004B2DB601C7010E9487118F5F9F4F29F44B2DB6018BE10E945111C7010E94CD3208
:2026A00028960FB6F894DEBF0FBECDBFCF91DF911F910F91FF90EF90DF90CF90BF9008952D
:2026C0002F923F924F925F926F927F928F929F92AF92BF92CF92DF92EF92FF920F931F9368
:2026E000DF93CF9300D000D0CDB7DEB76C01DC0112962D903C9013971596FC90BC016A5F6B
:202700007F4FDB0112968D919D910D90BC91A02D89839A83AB83BC83FB018681482E5524DC
:2027200066247724118190E00E948D32292F882E992E8114910459F48091C10080688093F8
:20274000C1004F2DB1018BE10E945111A0C0C6010D96442D50E0BC01882D922F0E940136A3
:202760008091C10080688093C10080914F078A3248F4883208F07FC08B3041F0873209F0DD
:202780007EC004C08B3209F07AC075C0112361F48091770290917802892B09F43FC081E44F
:2027A00092E00E94E82F3AC0113089F48091770290917802019721F087E492E00E94E82FD2
:2027C000A12C60EDB62E6AE1C62ED12C2DC0123089F48091770290917802029721F08DE4D3
:2027E00092E00E94E82FA12C50ECB52E58E1C52ED12C1AC0133009F042C0809177029091D6
:202800007802039721F085E592E00E94E82FA12C40EBB42E46E1C42ED12C06C0A12C30EE5D
:20282000B32E3CE1C32ED12C89819A81AB81BC812AE0B695A795979587952A95D1F761E07D
:202840000E949730109377021092780289819A81AB81BC81A80EB91ECA1EDB1EEE24E39452
:202860008401A3019201C601B5010E94A0284F2DB1018AE107C04F2DB1018DE103C04F2D7A
:20288000B1018BE10E945111C4010E94CD320F900F900F900F90CF91DF911F910F91FF9085
:2028A000EF90DF90CF90BF90AF909F908F907F906F905F904F903F902F9008951F93CF93D4
:2028C000DF93FC01C281D38115818091C10080688093C1000E94350688529A403CF4412F9D
:2028E000BE018BE10E9451118AE012C0412FBE018AE10E94511180E090EDAAE1B0E08093C4
:20290000540790935507A0935607B09357078AE280934F07DF91CF911F9108951F93CF93A6
:20292000DF93FC01C281D38115818091C10080688093C10080914F078A508230F8F40E94EC
:20294000350688529A404CF4412FBE018BE10E9451118AE080934F0716C080913607882307
:2029600011F085E205C08DE592E00E94E82F8BE280934F07412FBE018AE103C0412FBE012B
:202980008DE10E945111DF91CF911F910895EF92FF920F931F93CF93DF938C017B0150E035
:2029A00021E030E0C42FDD27C7FDD095BE01615070400BC0C901880F991F43E0220F331F3C
:2029C0004A95E1F7280F391F5F5F852F90E08617970784F350E040E302C040835F5F852FD3
:2029E00090E0F701E80FF91F8C179D07B4F3108240E017C080818F5F8083060F171F07C0E5
:202A0000F701E80FF91F66277727621B730B0217130784F7C9016AE070E00E9452369B01B1
:202A20004F5F842F90E08C179D0754F3DF91CF911F910F91FF90EF900895EF92FF920F93B8
:202A40001F93CF93DF93DC018B01E1E0F0E061E070E0E22EFF24E7FCF0940BC0CB01880F9D
:202A6000991F23E0660F771F2A95E1F7680F791F3196EE15FF0594F3E42FFF27E7FDF095F3
:202A8000EA0FFB1FC0E0D0E00DC08F5F020F131F06171707D0F78193CB016AE070E00E94B7
:202AA00052362196CE15DF0534F480E322273327261B370BEDCFDF91CF911F910F91FF90F4
:202AC000EF900895DF93CF930F92CDB7DEB78FB78983F89410926307109264071092650747
:202AE0001092660789818FBF80E090E00F90CF91DF9108950895CF92DF92EF92FF920F9370
:202B00001F93DF93CF930F92CDB7DEB76C01613011F48FEF3CC08FB78983F894E090630740
:202B2000F0906407009165071091660789818FBFC801B7012CE330E040E050E00E948736F8
:202B4000F6016283C801B7012CE330E040E050E00E948736CA01B9012CE330E040E050E056
:202B60000E948736F6016183C801B70120E13EE040E050E00E948736CA01B90128E130E02E
:202B800040E050E00E948736F601608380E00F90CF91DF911F910F91FF90EF90DF90CF90B1
:202BA0000895DF92EF92FF920F931F93DF93CF9300D000D0CDB7DEB76A837B838C83D72E15
:202BC000413011F48FEF30C0E82EFF24E7FCF0940F2D1F2D772767FD7095872F972F20E165
:202BE0003EE040E050E00E941F36E60EF71E081F191F8FB78983F8948CE32D2D2802C00176
:202C00001124AA2797FDA095BA2F8E0D9F1DA01FB11F8093630790936407A0936507B09329
:202C2000660789818FBF80E00F900F900F900F90CF91DF911F910F91FF90EF90DF900895B9
:202C40008FEF08958FEF08958091630790916407A0916507B09166070196A11DB11D8093B6
:202C6000630790936407A0936507B0936607089580914F05089580914D0590914E050E94F5
:202C800062300E94572B0E94982B10924E0510924D0510925005109251050895CF92DF92D2
:202CA000EF92FF920F931F93CF93DF93082FC0904D05D0904E0510915005C12FDD27C7FDA0
:202CC000D095CC0DDD1DF8808F2D90E00E94B036892B29F08F2D90E00E94B63688830230CC
:202CE00009F448C0033030F4002359F0013009F08DC020C0033009F444C0043009F086C00E
:202D000069C08881893389F18D3211F48FE230C08B32B9F0803411F48AE22AC08C3311F4ED
:202D20008EE326C08F35C9F0803211F481E420C08F5F1EC08881803211F489E319C08F3231
:202D400011F48DE215C08D3211F48BE211C08A3211F480E40DC08E3311F48CE309C08C3379
:202D600011F48FE505C0813411F480E201C0815088834CC011160CF058C0115010935005BC
:202D800054C0212F332727FD309580915105992787FD90950297281739070CF046C0212F52
:202DA0002F5F2093500580914F052817F1F5E22FFF27E7FDF095EC0DFD1D80E28083E22FCA
:202DC000EF5FE0934F05FF27E7FDF095EC0DFD1D10822BC040914F054150E42FFF27E7FDEC
:202DE000F0954F5FEC0DFD1D842F992787FD90950197D601A80FB91F20E030E0BC010CC0DA
:202E00008C911197803221F050934F0511E00EC01082215030403197542F520FCB01820FB8
:202E2000931F1816190664F3EFCF10E060914F0520915005E22EFF24E7FCF0946150E62FE3
:202E4000FF27E7FDF0956F5FEC0DFD1D862F992787FD90950197D601A80FB91F40E050E096
:202E6000EC0108C08C911197803261F41082415050403197762F740FCE01840F951FE8161A
:202E8000F90684F370934F05273014F400E002C0022F065080914F05992787FD909520915E
:202EA0005105C22FDD27C7FDD0952197C81BD90B202F332727FD3095BC01621B730B68303D
:202EC000710514F067E070E0802F992787FD90958C0D9D1D0E94203061E0CE010E9497300B
:202EE00080915005612F801B0E944E2FDF91CF911F910F91FF90EF90DF90CF900895AF9248
:202F0000BF92CF92DF92EF92FF920F931F93CF93DF936C01E62E80914D0590914E05892B48
:202F200009F092C081E0861708F08EC060935105D0924E05C0924D051092500510924F0573
:202F40008601C0E0D0E0A62EBB2412C08F2D90E00E94A236892B19F4E0E2FE1621F421960C
:202F60000F5F1F4F05C0C0934F05F801108209C0F801F080FF2019F0CA15DB053CF3C093E3
:202F80004F0580914F05882339F480E2F6018083118281E080934F0580914F058E1551F49C
:202FA000EE2DE150E0934F05FF27E7FDF095EC0DFD1D108240914F054150E42FFF27E7FDF7
:202FC000F0954F5FEC0DFD1D842F992787FD90950197D601A80FB91F20E030E0BC0108C0FC
:202FE0008C911197803261F41082215030403197542F520FCB01820F931F1816190684F313
:2030000050934F0580914F05C82FDD27C7FDD095BE01C830D10514F067E070E0C6010E945F
:203020002030C095D0958E2D992787FD909561E08C0F9D1F0E94973061E0809150050E9418
:203040004E2F20E030E002C02FEF3FEFC901DF91CF911F910F91FF90EF90DF90CF90BF90C0
:20306000AF900895FC0180819181828393830895FC01A281B3818C9111969C91828393834C
:203080000895FC01A281B38112968C91129713969C91828393830895FC01A281B381149645
:2030A0008C91149715969C91828393830895FC01A281B38116968C91169717969C9182830F
:2030C00093830895FC01828193810895FC0190E0848580FD05C09F5F0190F081E02DF8CF00
:2030E000892F0895FC0190E00280F381E02D848580FD02C09F5FF8CF892F0895FC018081AB
:2031000091810895FC01828193810895FC01808591850895FC0184858170089508950895CC
:2031200008950895089508950895089508950F931F93DF93CF930F92CDB7DEB78B0121E0D5
:203140002983DC011A96ED91FC911B97309719F0CE0101960995C8010E9486180E94E82FE3
:20316000D8011A96ED91FC911B97309721F01982CE01019609950F90CF91DF911F910F91D3
:203180000895FC018081823071F480913407882319F08EE792E002C085E892E00E94E82F3C
:2031A0008BE180934F070895FC01E081E13019F0E23001F511C080913A07882331F085B7F2
:2031C0008F7785BF85B78F7705C085B7806885BF85B7806885BF089580913A07882319F02B
:2031E0008EE792E002C085E892E00E94E82F8AE180934F070895FC018081823071F48091F7
:203200003707882319F08DE892E002C082E992E00E94E82F8DE180934F070895FC0180810B
:20322000813011F40E94572B0895EF92FF920F931F93DF93CF93CDB7DEB761970FB6F8947B
:20324000DEBF0FBECDBFFC01108144E050E069E972E07E010894E11CF11CC7010E94F2353C
:20326000113099F0113018F0123081F511C080914C07882319F080E090E003C0C7010E949D
:20328000DD1F61E00E94973021C00E94572B1EC080914C07882399F48E010B5F1F4F40E082
:2032A000B801C7010E94FA1D8F5F9F4F19F48DE992E007C0C8010E94623084E205C083EAA7
:2032C00092E00E94E82F8BE080934F0761960FB6F894DEBF0FBECDBFCF91DF911F910F9191
:2032E000FF90EF900895FC0180818230A1F480914C07882349F489EA92E00E94E82F0E9452
:2033000075268EEA92E002C083EA92E00E94E82F8BE080934F070895EF92FF920F931F93F7
:20332000DF93CF93CDB7DEB764970FB6F894DEBF0FBECDBFFC01108146E050E063EB72E0DA
:203340007E010894E11CF11CC7010E94F235113099F0113018F01230C9F517C080914C0769
:20336000882319F080E090E003C0C7010E94DD1F61E00E9497302AC081ED0E94E52B82E585
:203380000E94E52B0E94572B21C080914C078823B1F48E01085F1F4F40E0B801C7010E941B
:2033A000FA1D8F5F9F4F19F48DE992E00AC082E50E94CB2BC8010E94623081E205C089EBC3
:2033C00092E00E94E82F8BE080934F0764960FB6F894DEBF0FBECDBFCF91DF911F910F918D
:2033E000FF90EF900895FC01E081E130A9F0E13018F0E43018F513C08EE397E00E946230F1
:2034000080914D0790914E072FEF8F3F9207B1F060E00E94002E08950E94572B08958EE3CC
:2034200097E00E94623080914D0790914E072FEF8F3F920719F060E00E94002E08951F9319
:20344000DF93CF930F92CDB7DEB7FC0110811130A1F0113018F0123009F512C080914D07BE
:2034600090914E078F5F9F4FC9F060E080912F07909130070E94002E11C00E94572B0EC0CF
:203480008AE08983BE016F5F7F4F81E00E944F3382EC92E00E94E82F10934F070F90CF9145
:2034A000DF911F910895DF93CF9300D000D0CDB7DEB7FC01E081E130A1F0E13018F0E23097
:2034C00081F512C080914D0790914E078F5F9F4F41F160E080912F07909130070E94002E0C
:2034E00020C00E94572B1DC089E08983809131078A8380912F07909130079C838B83BE0195
:203500006F5F7F4F84E00E944F3382ED92E00E94E82F84E00E94CC300E94572B81E0809353
:203520004F070F900F900F900F90CF91DF910895FC01E081EE2319F0E130D9F411C080E0C5
:2035400090E00E94580724EF31E040E050E060E070E088E597E00E9400358093E2020895A7
:203560008091E2020E94AA3484EC0E94E52B0E94572B0895FC01E081E130B1F0E13018F0CA
:20358000E33081F51BC080E090E00E94580724EF31E040E050E060E070E088E597E00E946C
:2035A00000358093E30208958091E3020E94AA3484EC0E94E52B0E94572B089580E090E018
:2035C0000E9458078091E3020E94AA3424EF31E040E050E060E070E088E597E00E940035B5
:2035E0008093E3020895EF92FF920F931F93DF93CF93CDB7DEB72B970FB6F894DEBF0FBE66
:20360000CDBFFC01E081E13071F0E13018F0E23079F50CC08091310761E0992787FD9095F6
:203620000E94973025C00E94572B22C080913107992787FD90959093620780936107DE019E
:203640001196E4EEF2E08BE001900D928150E1F7E980FA800B811C812D813E814F815885B5
:2036600069857A858B850E94E91088E180934F072B960FB6F894DEBF0FBECDBFCF91DF9108
:203680001F910F91FF90EF900895EF92FF920F931F93DF93CF93CDB7DEB72B970FB6F894C9
:2036A000DEBF0FBECDBFFC01E081E13061F0E13018F0E23051F50AC061E080913D0790E013
:2036C0000E94973022C00E94572B1FC080913D078093610710926207DE011196EFEEF2E08C
:2036E0008BE001900D928150E1F7E980FA800B811C812D813E814F81588569857A858B8563
:203700000E94E91084E180934F072B960FB6F894DEBF0FBECDBFCF91DF911F910F91FF9089
:20372000EF900895E4E6F0E090819E7F9083206820937A00482B40937C0060937B0081E04C
:20374000809352051092530580E090E00895EAE7F0E080818F778083E4E6F0E08081816071
:2037600080831092520510925305089580915205882319F42FEF3FEF0AC081E080935305B4
:2037800080917A00806480937A0020E030E0C9010895982F80915305882399F080917A00C7
:2037A00086FD0FC01092530580917C009295990F907E892B80937C002091780030917900AD
:2037C00002C02FEF3FEFC9010895109255050895EF92FF920F931F93DF93CF93CDB7DEB788
:2037E0006C970FB6F894DEBF0FBECDBF7C01FC0160857185828593858E010F5F1F4F2CE193
:2038000030E040E050E00E9464296C3171058105910519F02FEF3FEF16C088899989AA8959
:20382000BB894096A11DB11DF70180839183A283B38384839583A683B783138A128A158A1E
:20384000148A20E030E0C9016C960FB6F894DEBF0FBECDBFCF91DF911F910F91FF90EF9079
:2038600008958F929F92AF92BF92CF92DF92EF92FF920F931F93DF93CF93CDB7DEB72897E3
:203880000FB6F894DEBF0FBECDBF5C014B01FC01C080D180E280F380C701B60120E132E043
:2038A00040E050E00E946536C61AD70AE80AF90A8E010F5F1F4F28E030E040E050E0C7012A
:2038C000B6010E94642989819A81AB81BC810097A105B10519F42FEF3FEF10C04096A11DC4
:2038E000B11DF50180839183A283B383F4018081918101969183808320E030E0C901289644
:203900000FB6F894DEBF0FBECDBFCF91DF911F910F91FF90EF90DF90CF90BF90AF909F90A7
:203920008F9008952F923F924F925F926F927F928F929F92AF92BF92CF92DF92EF92FF928D
:203940000F931F93DF93CF93CDB7DEB728970FB6F894DEBF0FBECDBF8D839E837A018B01E8
:2039600038872F83D90114968D919D910D90BC91A02D89839A83AB83BC83BC01CD0120E12D
:2039800032E040E050E00E9465365B016C01EF81F8852289922F990F80E09C0140E050E071
:2039A0002A0D3B1D4C1D5D1D6684778480889188D801C7014097A109B109820F931FA41FAD
:2039C000B51F681679068A069B0618F0170128010DC060E1262E312C412C512C260C371C6E
:2039E000481C591C221A330A440A550A89819A81AB81BC81E80EF91E0A1F1B1F40E1642E17
:203A000042E0742E812C912CC801B70120E132E040E050E00E94653679018A0169817A816D
:203A20008B819C8120E132E040E050E00E946536E216F3060407150709F467C06A187B087C
:203A40008C089D080D811E81A401930169817A818B819C810E946429AF81B88514962D91B5
:203A60003D914D915C911797260F371F481F591FFD01248335834683578362015101A61A20
:203A8000B70AC80AD90A32E1432E512C4A0E5B1E24E0E22EF12CEA0EFB1E3B014C012FC024
:203AA000B201C7010E94311C8F5F9F4F09F472C0A6019501317040705070AF81B88514962C
:203AC0006D917D918D919C9117970D811E810E946429EF81F8852481358146815781260F69
:203AE000371F481F591F2483358346835783660E771E881E991EA61AB70AC80AD90AA1143E
:203B0000B104C104D10461F61AC00D811E81A201910169817A818B819C810E946429EF8116
:203B2000F8852481358146815781260F371F481F591F248335834683578342013101EF81BD
:203B4000F885A480B580C680D780C601B50120E132E040E050E00E94653661157105810563
:203B60009105C1F480EF9DEFAFEFBFEFA80EB91ECA1EDB1EAF81B8851496AD92BD92CD9241
:203B8000DC9217975296B887AF83BD01CD010E970E94311CB301C40128960FB6F894DEBF6B
:203BA0000FBECDBFCF91DF911F910F91FF90EF90DF90CF90BF90AF909F908F907F906F90C6
:203BC0005F904F903F902F900895DF93CF9300D0CDB7DEB79C0142E050E060E070E0CE01E1
:203BE00001960E94921C89819A810F900F90CF91DF9108952F923F924F925F926F927F9298
:203C00008F929F92BF92CF92DF92EF92FF920F931F93DF93CF93CDB7DEB7A9970FB6F8944B
:203C2000DEBF0FBECDBFDC017B01B42E22E0421769F48CE190E0A0E0B0E08093FA0290937C
:203C4000FB02A093FC02B093FD028BC1FB011082FE01359620E030E0AE014F5F5F4F8C9118
:203C60008E3221F410821196FA0102C0882349F08C9181932F5F3F4F2C30310511F011960E
:203C8000EECF108280915405B816B9F18091FA029091FB02A091FC02B091FD0222E030E047
:203CA0001EC0BB2081F44C96A11DB11D8C30FBE09F07F0E0AF07F0E0BF0789F48CE190E0B5
:203CC000A0E0B0E00CC04C97A109B1098C319105A105B10520F480EF9AE0A0E0B0E0215094
:203CE00030404FEF2F3F3407E1F68093FA029093FB02A093FC02B093FD026090FA02709008
:203D0000FB028090FC029090FD02B0925405EEE0CE2ED12CCC0EDD1E76E1272E312C2C0EFF
:203D20003D1E2E010894411C511C6091FA027091FB028091FC029091FD0286012CE130E0D5
:203D400040E050E00E9464292091FA023091FB024091FC025091FD0289A19AA1ABA1BCA1BC
:203D600082179307A407B50759F1BB2079F0DA01C9014C97A109B1098C319105A105B10580
:203D8000B0F480EF9AE0A0E0B0E011C0DA01C9014C96A11DB11D8C30EBE09E07E0E0AE0701
:203DA000E0E0BE0721F48CE190E0A0E0B0E08093FA029093FB02A093FC02B093FD02D4C046
:203DC000BB2069F04C97A109B1098C319105A105B105A0F480EF9AE0A0E0B0E00FC04C967B
:203DE000A11DB11D8C30FBE09F07F0E0AF07F0E0BF0721F48CE190E0A0E0B0E08093FA02CD
:203E00009093FB02A093FC02B093FD028D818A3209F050C089818A3211F5F6019E012B5E51
:203E20003F4F8081882341F0D7018D937D01E217F30711F03196F5CFD7018EE28D93FE01BB
:203E400076969E01285E3F4F8081882309F488C08D93E217F30709F483C03196F5CF43E0B1
:203E600050E0B201C1010E941136009709F07CC0F6019E012B5E3F4F8081882341F0D70186
:203E80008D937D01E217F30711F03196F5CFD7018EE28D93FE0176969E01285E3F4F8081DE
:203EA000882309F45DC08D93E217F30709F458C03196F5CF48E050E0BE016B5F7F4FC60114
:203EC0000E941136009709F04FC089818A3201F5F6019E012B5E3F4F8081882341F0D7013C
:203EE0008D937D01E217F30711F03196F5CFD7018EE28D93FE0176969E01285E3F4F80817E
:203F0000882371F18D93E217F30751F13196F7CF43E050E0B201C1010E941136009721F554
:203F2000F6019E012B5E3F4F8081882341F0D7018D937D01E217F30711F03196F5CFD7012A
:203F40008EE28D93FE0176969E01285E3F4F8081882331F08D93E217F30711F03196F7CFA5
:203F60001C9220E030E010C08091FA029091FB02A091FC02B091FD0286159705A805B90577
:203F800009F0D3CE2FEF3FEFC901A9960FB6F894DEBF0FBECDBFCF91DF911F910F91FF903C
:203FA000EF90DF90CF90BF909F908F907F906F905F904F903F902F900895AF92BF92CF921D
:203FC000DF92EF92FF920F931F93DF93CF93CDB7DEB76A970FB6F894DEBF0FBECDBF6C0168
:203FE00042E07E010894E11CF11CB7010E94FA1D40E0B701C6010E94FA1D8F5F9F4F19F4C8
:2040000000E010E019C000E010E0FEE0AF2EB12CAC0EBD1E0F5F1F4F40E0B501C6010E94DF
:20402000FA1D8F5F9F4F41F04BE050E0B501C7010E941136009771F7C8016A960FB6F89481
:20404000DEBF0FBECDBFCF91DF911F910F91FF90EF90DF90CF90BF90AF9008954F925F9271
:204060006F927F928F929F92AF92BF92CF92DF92EF92FF920F931F93DF93CF93CDB7DEB725
:204080006A970FB6F894DEBF0FBECDBFDC01FE013E9620E030E0AE01495E5F4F8C918E3237
:2040A00021F410821196FA0102C0882349F08C9181932F5F3F4F2C30310511F01196EECFCD
:2040C00010820CE1C02ED12CE12CF12C15E0812E912C8C0E9D1EBEE04B2E512C4C0E5D1E2D
:2040E0005E010894A11CB11CA7E16A2E712C6C0E7D1E840128E030E040E050E0C701B601FD
:204100000E94642948E050E0B201C4010E9411360097A9F4C701B601685F7F4F8F4F9F4FA3
:20412000850123E030E040E050E00E94642943E050E0B301C5010E9411360097A9F08CE114
:2041400090E0A0E0B0E0C80ED91EEA1EFB1E9CE0C9169BE0D90690E0E90690E0F90649F62F
:20416000CC24CA94DC2C7601B601C7016A960FB6F894DEBF0FBECDBFCF91DF911F910F918C
:20418000FF90EF90DF90CF90BF90AF909F908F907F906F905F904F900895AF92BF92CF92FB
:2041A000DF92EF920F931F93DF93CF93CDB7DEB72C970FB6F894DEBF0FBECDBF60910706C4
:2041C000709108068091090690910A068E010B5F1F4F28E030E040E050E00E9464298D8173
:2041E0009E81AF81B8850097A105B10521F4AA24BB24650137C0A0900706B0900806C09046
:204200000906D0900A068093070690930806A0930906B0930A06EE24E39407E016E024E0CF
:2042200030E040E050E060E070E080E090E00E94A02819821A821B821C82609107067091E3
:2042400008068091090690910A066C5F7F4F8F4F9F4F8E010F5F1F4F24E030E040E050E0CB
:204260000E94A028B501C6012C960FB6F894DEBF0FBECDBFCF91DF911F910F91EF90DF9040
:20428000CF90BF90AF900895AF92BF92CF92DF92EF92FF920F931F93DF93CF93CDB7DEB7DD
:2042A000A5970FB6F894DEBF0FBECDBF8C010E942E206F5F7F4F8F4F9F4F09F08DC00E94AE
:2042C000CD205B016C01611571058105910509F483C0FE013A9620E030E0AE014E5E5F4FF8
:2042E000D8018C918E3229F410820F5F1F4FFA0102C0882359F0D8018C9181932F5F3F4FA6
:204300002C30310519F00F5F1F4FEACF10821D8A1E8A1F8A188E1DA2A98EBA8ECB8EDC8E3C
:20432000A9A2BAA2CBA2DCA21A821B821C821D821E821F8218861986EE24E3948E010E5F72
:204340001F4F28E030E040E050E0C601B5010E94A0288CE190E0A0E0B0E08D8F9E8FAF8F2C
:20436000B8A37E010894E11CF11C2AC0870121E030E040E050E00E9464298981AD8CBE8C2E
:20438000CF8CD8A0882381F4EE24E3948E01065F1F4F2CE130E040E050E0C601B5010E94B3
:2043A000A02820E030E01AC08CE190E0A0E0B0E0A80EB91ECA1EDB1EAD8EBE8ECF8ED8A292
:2043C0006D8D7E8D8F8D98A16C30ABE07A07A0E08A07A0E09A0750F22FEF3FEFC901A59616
:2043E0000FB6F894DEBF0FBECDBFCF91DF911F910F91FF90EF90DF90CF90BF90AF9008954F
:20440000DF92EF92FF920F931F93DF93CF93CDB7DEB76C970FB6F894DEBF0FBECDBF8C0101
:20442000D62E80915505882309F406C1C8010E942E206C8B7D8B8E8B9F8B6F3F2FEF72075E
:204440002FEF82072FEF920709F474C08E010F5F1F4F2CE130E040E050E00E946429EC8852
:20446000FD880E891F89E8E9F5E00AC080859185A285B3858E159F05A007B10731F07696BB
:2044800086E0E630F80791F702C0309739F420910606622F70E040E050E007C084858D21F7
:2044A00080FDCAC081FDC8C0C9C0CB01042E02C0959587950A94E2F780FD0CC081E090E0CF
:2044C000042E02C0880F991F0A94E2F7282B2093060607C04F5F5F4F4930510531F74FEFB8
:2044E0005FEF642F4F3F09F4A7C0242F332727FD309586E190E0289FF001299FF00D389F28
:20450000F00D1124EA5AFA4F458788899989AA89BB894096A11DB11D80839183A283B38392
:2045200084839583A683B783D486E086F186028713876FC0D4FE80C0C8010E9444218F5FA0
:204540009F4F09F479C0C8010E942E206F3F2FEF72072FEF82072FEF920709F46DC06C8BBA
:204560007D8B8E8B9F8B8E010F5F1F4F2CE130E040E050E00E94642920910606622F70E04B
:2045800040E050E0CB01042E02C0959587950A94E2F780FD0CC081E090E0042E02C0880FA9
:2045A000991F0A94E2F7282B2093060607C04F5F5F4F4930510531F74FEF5FEF642F4F3FF3
:2045C000D9F1242F332727FD309586E190E0289FF001299FF00D389FF00D1124EA5AFA4F91
:2045E000458788899989AA89BB894096A11DB11D80839183A283B38384839583A683B783EF
:20460000D4868C899D89AE89BF8980879187A287B3878C859D85AE85BF8586879787A08B04
:20462000B18B138A128A158A148A86E16802F0011124EA5AFA4F02C0E0E0F0E0CF016C9620
:204640000FB6F894DEBF0FBECDBFCF91DF911F910F91FF90EF90DF9008952F923F924F9266
:204660005F926F927F928F929F92AF92BF92CF92DF92EF920F931F93DF93CF93CDB7DEB7BF
:2046800028970FB6F894DEBF0FBECDBF1C01DC01AD90BD90CD90DC900E94CD202B013C01CF
:2046A000611571058105910519F42FEF3FEF50C0C601B50120E132E040E050E00E9465366C
:2046C000A61AB70AC80AD90A19821A821B821C82AD82BE82CF82D8864E010894811C911CDF
:2046E000EE24E394840128E030E040E050E0C301B2010E94A02828E030E040E050E0C60134
:20470000B5010E94642949825A826B827C8228E030E040E050E0C601B5010E94A02880E172
:2047200090E0A0E0B0E0480E591E6A1E7B1ED1014D925D926D927C92139754968D919C917F
:204740005597019655969C938E93549720E030E0C90128960FB6F894DEBF0FBECDBFCF9171
:20476000DF911F910F91EF90DF90CF90BF90AF909F908F907F906F905F904F903F902F90E6
:2047800008952F923F924F925F926F927F928F929F92AF92BF92CF92DF92EF92FF920F939C
:2047A0001F93DF93CF93CDB7DEB727970FB6F894DEBF0FBECDBF49835A836B837C833F83FD
:2047C0002E832C01D9016D907D908D909C90CB01BA01660D771D881D991D20E132E040E0B2
:2047E00050E00E94653679018A01C401B30120E132E040E050E00E946536E216F306040732
:20480000150709F48AC0C401B30120E132E040E050E00E946536B0E1AB2EB2E0BB2EC12C4A
:20482000D12CA61AB70AC80AD90AEE24E3948201A6019501C401B3010E94A028660E771E10
:20484000881E991EEE81FF81608271828282938269807A808B809C806A187B088C089D08D6
:2048600012012A0C3B1CA4E14A2E512C4E0E5F1EED83FF804BC0AE81BF8154962D913C9167
:204880005597442737FD4095542F1E968D919D910D90BC91A02D79E0B695A7959795879556
:2048A0007A95D1F7281739074A075B0730F4B2018D819F2D0E94311C04C08E819F810E94BA
:2048C0002D23EE81FF81A080B180C280D380A4019301317040705070EE24E3948101C60197
:2048E000B5010E94A028A60EB71EC81ED91EAE81BF81AD92BD92CD92DC92139780E09EEFD1
:20490000AFEFBFEF682279228A229B22611471048104910409F0AFCF16C0EE24E394820160
:2049200029813A814B815C81C401B3010E94A028660E771E881E991EAE81BF816D927D92A3
:204940008D929C921397EE81FF81E080F18002811381C801B70120E132E040E050E00E9403
:204960006536611571058105910599F580EF9DEFAFEFBFEFE80EF91E0A1F1B1FAE81BF81E0
:20498000ED92FD920D931C93139754962D913C915597442737FD4095542FFD018685978593
:2049A000A089B18969E0B695A795979587956A95D1F7281739074A075B0738F4BF016C5ECD
:2049C0007F4FCF010E94311C04C08E819F810E942D23AE81BF816D917D918D919C9120E19E
:2049E00032E040E050E00E9465366051704080409040AE81BF815496EC9154973E2F330FB7
:204A000020E040E050E0260F371F481F591FFD0126873787408B518B69817A818B819C81BE
:204A200027960FB6F894DEBF0FBECDBFCF91DF911F910F91FF90EF90DF90CF90BF90AF90E8
:204A40009F908F907F906F905F904F903F902F900895DF93CF930F92CDB7DEB789839B01CB
:204A600041E050E060E070E0CE0101960E94C123CB010F90CF91DF910895EF920F931F93BC
:204A8000CF93DF93EC01409106068D85282F332727FD3095842F90E0022E02C09595879571
:204AA0000A94E2F780FF35C081E090E002C0880F991F2A95E2F780958423809306062097FF
:204AC00041F18E01025F1F4F688579858A859B85655F7F4F8F4F9F4FEE24E39424E030E031
:204AE00040E050E00E94A0281C86188219821A821B821C821D821E821F828FEF9FEFAFEFC4
:204B0000BFEF88879987AA87BB871D8620E030E002C02FEF3FEFC901DF91CF911F910F919A
:204B2000EF900895AF92BF92CF92DF92EF92FF920F931F93DF93CF93CDB7DEB7A5970FB6A1
:204B4000F894DEBF0FBECDBF0E942E205B016C018CE0A8168BE0B80680E0C80680E0D8065B
:204B6000B9F0E8E9F5E00AC080859185A285B3858A159B05AC05BD0531F0769686E0E63047
:204B8000F80791F708C0309731F0CF010E943D252FEF3FEF6EC08E01065F1F4F2CE130E011
:204BA00040E050E0C601B5010E94642960910B0670910C0680910D0690910E06EE24E39402
:204BC0008E01075E1F4F24E030E040E050E00E94A028898D9A8DAB8DBC8D80930B069093A0
:204BE0000C06A0930D06B0930E0612E0E12EF12CEC0EFD1E60910B0670910C0680910D069A
:204C000090910E06870128E030E040E050E00E9464298A819B81AC81BD810097A105B105BB
:204C200029F0582F492F3A2F2B2F08C050910B0640910C0630910D0620910E0650930B066F
:204C400040930C0630930D0620930E060097A105B10581F61982EE248E010F5F1F4F2CE143
:204C600030E040E050E0C601B5010E94A02820E030E0C901A5960FB6F894DEBF0FBECDBF91
:204C8000CF91DF911F910F91FF90EF90DF90CF90BF90AF9008950F931F930E944B07EEE5D2
:204CA000F5E08FEF9FEFAFEFBFEF80839183A283B383769626E0EE30F207B9F787E0809302
:204CC000060607E016E024E030E040E050E060E070E080E090E00E94642981E0809355052A
:204CE00080E090E01F910F9108958F929F92AF92BF92CF92DF92EF920F931F93DF93CF9398
:204D0000CDB7DEB729970FB6F894DEBF0FBECDBF1982EE248E010F5F1F4F20EF3AE040E012
:204D200050E06CE170E080E090E00E94A02880E890E1A0E0B0E08093070690930806A093FF
:204D40000906B0930A06EE24E39407E016E024E030E040E050E060E070E080E090E00E9425
:204D6000A02880E395E0A4E0B0E080930B0690930C06A0930D06B0930E0624E030E040E055
:204D800050E064E070E080E090E00E94A02880E992E1A0E0B0E08A839B83AC83BD8380E728
:204DA0009EE0A0E0B0E08E839F83A887B98780E8A82E80E1B82EC12CD12C02E0802E912C07
:204DC0008C0E9D1EEE24E394840128E030E040E050E0C601B5010E94A0288A819B81AC81CD
:204DE000BD81805F9D4FAF4FBF4F8A839B83AC83BD838E819F81A885B985805F9D4FAF4FA1
:204E0000BF4F8E839F83A887B98780E192E0A0E0B0E0A80EB91ECA1EDB1E90E4A91697E0E7
:204E2000B90694E0C90690E0D90661F660910706709108068091090690910A0628E030E054
:204E400040E050E00E9464291E821F821886198660910706709108068091090690910A06F7
:204E600028E030E040E050E00E94A02860910B0670910C0680910D0690910E0628E030E0DA
:204E800040E050E00E9464291A821B821C821D8260910B0670910C0680910D0690910E06AF
:204EA00028E030E040E050E00E94A028109255050E944B2680E090E029960FB6F894DEBF94
:204EC0000FBECDBFCF91DF911F910F91EF90DF90CF90BF90AF909F908F900895E4E6F0E0F9
:204EE00090819B7F908323982B9894B1976094B9289AE22FF0E0E470F070F595E795F59586
:204F0000E795E068EDBD10921406109213061092120610921106109216061092150610921C
:204F2000100610920F0610921706682B642B60642370622B6CBD80E090E00895E4E6F0E0AF
:204F40008081846080830895FC0180911706882319F02FEF3FEF20C08DB580688DBD80814C
:204F60008EBDDB019A0108C00DB407FEFDCF9EB581818EBD9D93319621503040A9F7FA0102
:204F80003197E60FF71F0DB407FEFDCF8EB580831092170620E030E0C90108958091170602
:204FA000089580911A0690911B0608958091180690911906089582E296E027ED209322066F
:204FC00010922306289842E050E0BC010E943207289A80912306089583E88093220620916C
:204FE00018063091190680E190E0821B930BAB0102C0569547958A95E2F740932306285006
:20500000304002C0660F771F2A95E2F76093240610922506289844E050E062E276E0CB0157
:205020000E943207289A0E94DB278C7B8C3AD9F7089583E5809322062091180630911906A3
:2050400080E190E0821B930BAB0102C0569547958A95E2F7409323062850304002C0660FFC
:20506000771F2A95E2F76093240610922506289844E050E062E276E0CB010E943207289A01
:205080000E94DB278C7B8C3AD9F708959F92AF92BF92CF92DF92EF92FF920F931F93DF93C5
:2050A000CF930F92CDB7DEB75A017901902E84E88093220610922306709324066093250684
:2050C000289844E050E062E276E0CB010E94320700E010E06E010894C11CD11C0DC041E0E8
:2050E00050E0B601C7010E943207992019F00894E11CF11C0F5F1F4F0A151B0580F3289A6E
:205100000F90CF91DF911F910F91FF90EF90DF90CF90BF90AF909F90089582E296E024E8B4
:2051200020932206109223067093240660932506289844E050E0BC010E943207289A089573
:205140002F923F924F925F926F927F928F929F92AF92BF92CF92DF92EF92FF920F931F93BD
:20516000DF93CF9300D000D000D0CDB7DEB72B013C0129833A834B835C8318011E2DC90125
:20518000DA014C015D0158C0C301B20120E132E040E050E00E94653669017A01C501B401FA
:2051A000640D751D861D971D20E132E040E050E00E9465362C153D054E055F0579F0C3018E
:2051C000B20120E132E040E050E00E94653620E132E0261B370B3E832D8302C09E828D8284
:2051E000B60181E00E941928B60181E00E948D28C301B20120E132E040E050E00E9465362E
:20520000012F91014D815E8181E00E944628B60181E00E94EC27ED81FE81CF01A0E0B0E014
:20522000112311F02E0E3F1E480E591E6A1E7B1E881A990AAA0ABB0A81149104A104B10470
:2052400009F0A2CF69817A818B819C8126960FB6F894DEBF0FBECDBFCF91DF911F910F91B3
:20526000FF90EF90DF90CF90BF90AF909F908F907F906F905F904F903F902F900895EF92EE
:20528000FF920F931F938A01790182E296E024ED2093220610922306709324066093250648
:2052A00010922606289845E050E0BC010E943207A801B70186E296E00E943207289A1F91E7
:2052C0000F91FF90EF9008952F923F924F925F926F927F928F929F92AF92BF92CF92DF9257
:2052E000EF92FF920F931F93DF93CF9300D000D0CDB7DEB73B014C01322E232E49835A83D8
:205300002801C901DA015C016D014FC0C401B30120E132E040E050E00E94653679018A01C7
:20532000C601B501660D771D881D991D20E132E040E050E00E9465362E153F0540075107C8
:2053400079F0C401B30120E132E040E050E00E94653620E132E0261B370B3C832B8302C006
:20536000BC82AB82B70181E00E941928C401B30120E132E040E050E00E94653692014B814E
:205380005C8181E00E943F29EB81FC81CF01AA2797FDA095BA2F680E791E8A1E9B1EA81A59
:2053A000B90ACA0ADB0A4E0E5F1EA114B104C104D10409F0ABCF632D722D89819A810F902E
:2053C0000F900F900F90CF91DF911F910F91FF90EF90DF90CF90BF90AF909F908F907F9009
:2053E0006F905F904F903F902F900895E2E2F6E022ED20932206409118065091190620E141
:2054000030E0241B350BDC0102C0B695A7952A95E2F7A09323064850504002C0880F991FAA
:205420004A95E2F7780F7093240660932506289848E050E0BF01CF010E943207289A089500
:20544000E2E2F6E023E020932206409118065091190620E130E0241B350BDC0102C0B6956B
:20546000A7952A95E2F7A09323064850504002C0880F991F4A95E2F7780F70932406609364
:205480002506289848E050E0BF01CF010E943207289A089582E296E027ED20932206109294
:2054A0002306289842E050E0BC010E943207289A80912306807808950E9440072C982C9A15
:2054C000E2E2F6E001C0119286E0EA32F807D9F70E94DB2790E0FC01E873F07043E0F69503
:2054E000E7954A95E1F7EE0FFF1FEE0FFF1FDF01AA54BC4F2D913C9130931906209318061C
:20550000E854FC4F2081318130931B0620931A068C7390708C9719F02FEF3FEF02C020E0C1
:2055200030E0C9010895EFE7F0E080818E7F80836A98729A81988998EC9AEBE6F0E08081CD
:205540008460808380E090E00895EFE7F0E0808181608083EC98EBE6F0E080818B7F808339
:2055600008951F920F920FB60F9211240F900FBE0F901F901895CF93DF9327E040E460E0FB
:2055800081E00E94921B0E94B61B80E00E94C91BEC018FEFCF3FD807C1F30E94A71B83E02F
:2055A000C137D80714F080E012C082E0C138D80714F082E00CC081E0C138D80714F084E0D1
:2055C00006C0C13CD10514F481E001C088E0629B8061DF91CF910895E4E6F0E080818061D9
:2055E000808310922C060895DF93CF9300D000D00F92CDB7DEB749835A836B837C838D8363
:20560000282F80912C06882319F42FEF3FEF17C09091E40020937A0610927B068A818F63BD
:205620008093E5008B818093E6008C818093E70098788981982B9093E40020E030E0C901A8
:205640000F900F900F900F900F90CF91DF910895DF93CF93CDB7DEB72A970FB6F894DEBF26
:205660000FBECDBF8091E5008A838091E6008B838091E7008C838091E4008983DE01169636
:20568000FE01319685E001900D928150E1F72E813F81488559856A8570E090E02A960FB6B8
:2056A000F894DEBF0FBECDBFCF91DF9108956091FE027091FF0280912C06882339F140E0D0
:2056C00050E020C08D91282F2F71FB01E20FF11D208182958695877090E0032E02C0880FE6
:2056E000991F0A94E2F780958223808384E0AF36B80741F74E5F5F4F4830510519F420E048
:2057000030E006C0342FA8E6B4E0DCCF2FEF3FEFC9010895982F80912C06882319F42FEFF0
:205720003FEF04C09093850620E030E0C9010895109284060895982F6091FE027091FF02CF
:2057400080912C06882319F42FEF3FEF22C0492F552747FD5095440F551FA8E6B4E08D91FC
:20576000282F2F71FB01E20FF11D208182958695877090E0042E02C0880F991F0A94E2F743
:2057800080958223808384E0AF36B80741F720E030E0C9010895382F8091FE029091FF02FB
:2057A000232F2F71243180F4FC01E20FF11D208132953695377081E090E002C0880F991F76
:2057C0003A95E2F7282B20830895382F8091FE029091FF02232F2F71243188F4FC01E20F43
:2057E000F11D208132953695377081E090E002C0880F991F3A95E2F78095822380830895DD
:20580000EF92FF920F931F93CF93DF93E82F9B01682F70E0C901860F971F839720F022E271
:2058200030E0261B370BDB01A159BB4F40E050E0CE2FD0E0620F731F01E010E01BC08C912C
:205840002091FE023091FF02982F9F71943178F4F901E90FF11D208182958695877078018A
:2058600002C0EE0CFF1C8A95E2F72E2920834F5F5F4F1196CA018C0F9D1F86179707FCF211
:20588000DF91CF911F910F91FF90EF900895EF92FF920F931F93CF93DF93E82F9B01682FB9
:2058A00070E0C901860F971F839720F022E230E0261B370BDB01A159BB4F40E050E0CE2F95
:2058C000D0E0620F731F01E010E01DC08C912091FE023091FF02982F9F71943188F4F901C5
:2058E000E90FF11D2081829586958770780102C0EE0CFF1C8A95E2F7C7018095822380830B
:205900004F5F5F4F1196CA018C0F9D1F86179707ECF2DF91CF911F910F91FF90EF9008957E
:205920001F93DF93CF9300D000D00F92CDB7DEB749835A836B837C838D83182F80912C0657
:20594000882339F08091640080618093640010922C06809164008F7E809364008A818F63DC
:205960008093E5008B818093E6008C818093E700898188688093E40062E270E080E00E949C
:20598000472C10937A0610927B06109378061092790688E090E090938306809382069093CA
:2059A00081068093800690937F0680937E0690937D0680937C068FE0809385061092860612
:2059C00081E080932C0680E090E00F900F900F900F900F90CF91DF911F9108950F931F93C5
:2059E000CF93DF93282FC091FE02D091FF0280918D0690E0062E02C0959587950A94E2F702
:205A000080FD20E0660F771FA8E6B4E040E050E0022F10E0C801042E02C0959587950A94CA
:205A2000E2F79C9180FF14C0892F8F71FE01E80FF11D2081929596959770892F90E0062EFB
:205A400002C0880F991F0A94E2F7282B208314C0892F8F71FE01E80FF11D20819295969545
:205A60009770892F90E0062E02C0880F991F0A94E2F78095822380834F5F5F4F1196473004
:205A8000510541F6DF91CF911F910F910895AF92BF92CF92DF92EF92FF920F931F93CF9390
:205AA000DF937C01D62EC42E90938A068093890640938B0660938C06C0E0D0E000E010E0A3
:205AC0002FE0A22EB12CF501002E02C0EE0FFF1F0A94E2F7EE21FF21002E02C0F695E7956C
:205AE0000A94E2F7EA5AFB4FBE0180810E94EE2C2196C430D10509F441C00C5F1F4FC70105
:205B0000002E02C0969587950A94E2F7892BD9F6BE01DD20B1F02196CC2019F0E1E1F0E0B9
:205B200002C0E0E0F0E0EA5AFB4F80810E94EE2CCC2001F5E091FE02F091FF028085806806
:205B400006C0E091FE02F091FF0280858F77808711C0CC2019F0E0E1F0E002C0E0E0F0E0D1
:205B60008E010F5F1F4FEA5AFB4FBE0180810E94EE2CE801C430D10564F30CC0E091FE0269
:205B8000F091FF02DD2019F08085806802C080858F77808780E090E0DF91CF911F910F91CC
:205BA000FF90EF90DF90CF90BF90AF900895282F80912C06882319F42FEF3FEF1FC0809150
:205BC0008506922F98239093860662238095862B80938D0680918206909183069093810631
:205BE0008093800640918B0660918C068091890690918A060E94472D20E030E0C901089549
:205C00009C01462F80912C06882319F42FEF3FEF05C060E0C9010E94472D9C01C901089542
:205C200040918B0660918C068091890690918A060E94472D08950F931F93CF93DF93E82F3C
:205C40002091FE023091FF026730710508F053C080528B3508F04FC0E13608F0EF7D8E2FE8
:205C60008052813408F047C0E82FF0E0EE0FFF1FEA52FC4FC081D181862F86958901080F11
:205C8000111DE8E0F0E440E050E06F5F7F4F61707070D801A40FB51FCE018F70382F9E2F3B
:205CA0009F7024E0D695C7952A95E1F784E0F695E7958A95E1F76115710519F0292F206F35
:205CC00006C03295307F292F2295207F2F609C918C91832B9223892B8C938C919C91282336
:205CE000232B29232C934B5F5F4F4431510589F620E030E002C02FEF3FEFC901DF91CF91F1
:205D00001F910F910895CF92DF92EF92FF920F931F93CF93DF936C018B01C0E0D0E005C07C
:205D2000BE0180E20E941B2E2196C017D107C4F351E7E52E56E0F52EE00EF11EE80113C0DD
:205D4000F6018081F7018083882319F4BE0180E204C00894C11CD11CBE010E941B2E2196EC
:205D60000894E11CF11CC730D10554F380E090E0DF91CF911F910F91FF90EF90DF90CF909D
:205D8000089580917006882379F120912A0630912B06F901E15DF94F8081882339F41092FC
:205DA0002B0610922A0686E090E007C08091000390910103009731F0019790930103809380
:205DC000000306C02F5F3F4F30932B0620932A06609100037091010380912A0690912B067B
:205DE000815D994F0E94832E08950F931F93982F80912C06882319F42FEF3FEF26C0009114
:205E00002D0610912E06F801E15DF94F90830F5F1F4F10932E0600932D06F801E15DF94FF0
:205E2000108280912A0690912B0660E070E0815D994F0E94832E10927006083011051CF022
:205E400081E08093700620E030E0C9011F910F9108958091880660918706882369F0E62F5B
:205E6000FF27E7FDF095BF01EF58F94F80810E941B2E109288060895772767FD7095FB0188
:205E8000EF58F94F8081803211F080E201C08FE50E941B2E81E0809388060895982F873020
:205EA00018F02FEF3FEF13C06093880681E080938406909387060E94292F80917E069091DC
:205EC0007F0690937D0680937C0620E030E0C90108951F920F920FB60F9211242F933F930A
:205EE0004F935F936F937F938F939F93AF93BF93EF93FF93809170068823D1F0809178063C
:205F00009091790601979093790680937806892B61F560E070E081EC97E00E948B31809129
:205F20007A0690917B0690937906809378061DC0809184068823C9F080917C0690917D06F9
:205F4000019790937D0680937C06892B71F460E070E08EEB97E00E948B3180917E069091C1
:205F60007F0690937D0680937C06209186062223F1F080918006909181060197909381067D
:205F800080938006892B99F480918D06822780938D0660E070E08BEB97E00E948B31809148
:205FA0008206909183069093810680938006FF91EF91BF91AF919F918F917F916F915F917C
:205FC0004F913F912F910F900FBE0F901F9018950F931F93CF93DF93EC0180912C068823E7
:205FE00019F42FEF3FEF26C010927006CE010E94E9358C01AC014F5F5F4FBE018FE296E07F
:206000000E94F23510932E0600932D0610922B0610922A0660E070E08FE296E00E94832EAB
:2060200010927006083011051CF081E08093700620E030E0C901DF91CF911F910F9108956D
:20604000EF92FF920F931F93CF93DF93282F7B0180912C06882319F42FEF3FEF2BC010925F
:206060007006EB016134710514F0C0E4D0E00FE216E0AE01622F792FC8010E940136C00F1B
:20608000D11F1882F0922E06E0922D0610922B0610922A0660E070E0C8010E94832E109228
:2060A000700688E0E816F1041CF081E08093700620E030E0C901DF91CF911F910F91FF9090
:2060C000EF9008950F931F938C0180912C06882319F42FEF3FEF27C0B8018FE296E00E9453
:2060E0000A36F801D8010D900020E9F78D01015010400E1B1F0B10932E0600932D06109230
:206100002B0610922A0660E070E08FE296E00E94832E10927006083011051CF081E08093CC
:20612000700620E030E0C9011F910F910895EF92FF921F93CF93DF939C01162F80912C0665
:20614000882319F42FEF3FEF1FC088ED213F380714F421EF38EDE90187E22031380714F024
:20616000CFE0D7E2CE01D7FF04C0882799278C1B9D0B0E946C067E016F2D661F6627661FCA
:20618000412F0E94472D9C01C901DF91CF911F91FF90EF9008950895813099F0813018F057
:2061A000833099F51CC08091B00088678093B0008091700082608093700080EA8093B30039
:2061C0000BC0809170008D7F809370008091B0008F7C8093B0002F9A10928E0608958091A8
:2061E000B00088678093B0008091700082608093700080EA8093B30088E090E09093920694
:206200008093910681E080938E0608952F9A279A2F9A81E00E94CC3080E090E008951F92BF
:206220000F920FB60F9211242F933F938F939F9380918E06882339F180918F069091900663
:2062400001979093900680938F060196E1F48091020390E021E030E08227932780930203C7
:20626000882321F48091B0008F7C03C08091B00080638093B00080919106909192069093E4
:20628000900680938F069F918F913F912F910F900FBE0F901F901895809888986F9A779829
:2062A00080E090E008950895259A2D986F9A779880E090E00895089580E090E0089510921F
:2062C000930608958FEF9FEF08951092680783E1809394061092670784E18093BA071092D2
:2062E000B90781E00895DF93CF930F92CDB7DEB78FB78983F8941092680783E18093940652
:206300001092670784E18093BA0789818FBF0F90CF91DF910895DF93CF930F92CDB7DEB742
:206320003091BA07332311F480E024C020916807E22FF0E0EE0FFF1FEE0FFF1FE759F84F7E
:2063400091838083738362838FB78983F894233119F41092680703C02F5F20936807809177
:2063600067078F5F8093670731503093BA0789818FBF81E00F90CF91DF910895DF93CF93A2
:206380000F92CDB7DEB78FB78983F89490916707992319F489818FBF27C08091940683316F
:2063A00019F41092940603C08F5F809394069150909367078091BA078F5F8093BA07898126
:2063C0008FBF80919406E82FF0E0EE0FFF1FEE0FFF1FE759F84F208131812115310521F050
:2063E00082819381F90109950F90CF91DF91089510929506109297061092960681E008952A
:20640000CF92DF92EF92FF920F931F93DF93CF930F92CDB7DEB78C01D901009709F472C089
:20642000423008F46FC06230710508F46BC08FB78983F894F8019801260F371F50E0C42E73
:20644000DD2476010894E108F10806C031832083F901260F371F5F5F852F90E08E159F057B
:20646000ACF31182108211967C936E9312964C93129713964C93139715961C930E93149799
:20648000C69EC001C79E900DD69E900D11240197800F911F17969C938E93169719961C93B0
:2064A0000E93189750919506552349F41B961C921E921A97B0939706A09396061CC0E0919F
:2064C0009606F09197068F01452F808191818617970740F42285338541508F0121F0C90121
:2064E000FC01F3CF9F01F801B387A2871A962C931A971B963C935F5F5093950689818FBFAD
:2065000081E001C080E00F90CF91DF911F910F91FF90EF90DF90CF900895DF93CF930F924C
:20652000CDB7DEB7AC01009789F120919506222369F18FB78983F894E0919606F091970690
:20654000808191818417950728F08381882311F081E005C00284F385E02D215080E02223E2
:2065600019F0882369F305C0882319F4A0E0B0E00AC0A085B1858D919C9111979187808747
:2065800083818150838389818FBF02C0A0E0B0E0CD010F90CF91DF910895DF93CF930F92A7
:2065A000CDB7DEB7DC01009799F140919506442379F18FB78983F894E0919606F09197067E
:2065C0002681378184819581A817B90728F02A173B0710F081E005C00284F385E02D415065
:2065E00080E0442319F0882359F302C0882371F093818281981760F48085918511969C93FB
:206600008E93B187A08783818F5F838389818FBF0F90CF91DF910895982F882399F161152C
:20662000710581F14115510569F18091C1008F778093C1001092BB071092980670939B0678
:2066400060939A0690939D0650939F0640939E06809164008D7F8093640088E18093C000AE
:206660008093C10086E08093C20081E090E09093C5008093C4008091C10080688093C100ED
:2066800081E0089580E00895E1ECF0E080818F778083E4E6F0E08081826080830895482FC4
:2066A000FB012FEF3FEF02C0215030408091C00085FD04C021153105B9F758C0232B09F459
:2066C00055C082E08093C60057E19081923051F0973141F0933031F02FEF3FEF25C021509F
:2066E000304002C02FEF3FEF8091C00085FD04C021153105A1F73AC0232BC1F15093C6005E
:206700002FEF3FEF02C0215030408091C00085FD04C021153105B9F729C02115310531F1E0
:2067200090640DC0215030408091C00085FD04C021153105B9F71AC021153105B9F0909372
:20674000C600415021F03196C0CF215030408091C00085FD04C021153105B9F707C0232B52
:2067600029F083E08093C60081E0089580E00895DF93CF930F92CDB7DEB71092BB07109235
:2067800098061092990610929C0603C08091C60089838091C00087FDF9CF8091C100806859
:2067A0008093C1000F90CF91DF9108951F920F920FB60F9211242F933F934F938F939F9342
:2067C000AF93BF93EF93FF938091C00083FF07C08091B9078F5F8093B90710929906909103
:2067E000C60080919906882319F4923009F068C040919C0680919D06481708F061C0923027
:2068000031F41092980681E0809399060BC09330D9F53091BA07332341F48091B9078F5FD8
:206820008093B90710929C064BC020916807E22FF0E0EE0FFF1FEE0FFF1FDF01A759B84F18
:2068400080919E0690919F068D939C93E559F84F80919A0690919B0691838083233119F4FE
:206860001092680703C02F5F2093680731503093BA07809167078F5F809367078091C100CF
:206880008F778093C1001CC0973121F481E08093980616C080919806E0919A06F0919B069B
:2068A000242F30E0882319F4E20FF31F05C010929806E20FF31F9F7B90834F5F40939C0662
:2068C000FF91EF91BF91AF919F918F914F913F912F910F900FBE0F901F901895A0E7B0E0DA
:2068E0008C918E7F8C931092BC071092BD071092BE071092BF071092B200E6EBF0E08081BF
:20690000886080838C9181608C93E0EBF0E08081887F808380818160808380E090E0089577
:20692000DF93CF930F92CDB7DEB78FB78983F89489818FBF6091BC077091BD078091BE0744
:206940009091BF070F90CF91DF91089580E090E008950895982F81508730B8F4892F9927C7
:2069600087FD9095FC01EE0FFF1FE80FF91FEE0FFF1FEE0FFF1FE056F94F80819181892BCC
:2069800021F01182108280E008958FEF0895EF92FF920F931F93CF93DF937B018C01C0EABC
:2069A000D6E02881398121153105F1F088859985AA85BB85E816F9060A071B07A8F06A8124
:2069C0007B81C9010E948B3188859985AA85BB852C813D814E815F81820F931FA41FB51F05
:2069E00088879987AA87BB872C9687E0C030D807C1F6DF91CF911F910F91FF90EF9008957B
:206A00005F926F927F928F929F92AF92BF92CF92DF92EF92FF920F931F93CF93DF934C0136
:206A20003B0179018A010E9490345B016C01E0EAF6E0C0E0D0E05C2E80819181892BB1F5FF
:206A400087E0EE0CFF1C001F111F8A95D1F7C801B70128EE33E040E050E00E946536C90183
:206A6000DA01FE01EE0FFF1FEC0FFD1FEE0FFF1FEE0FFF1FAF014056594FEA0199828882D6
:206A80009F012E55394FE90179826882EC55F94F80839183A283B3838A0D9B1DAC1DBD1D8F
:206AA000FA0180879187A287B38708C021963C96C830D10509F0BFCF55245A94852DDF912A
:206AC000CF911F910F91FF90EF90DF90CF90BF90AF909F908F907F906F905F900895FC01B7
:206AE0008491089581E008950895DF93CF930F92CDB7DEB79C018FB78983F894F999FECFE1
:206B000032BD21BDF89A80B599819FBF0F90CF91DF91089508950895DF93CF930F92CDB72A
:206B2000DEB78FB78983F89407B600FCFDCF89E0E0E0F0E080935700849199819FBF0F90CE
:206B4000CF91DF910895DF93CF930F92CDB7DEB78FB78983F89407B600FCFDCF89E0E3E0AB
:206B6000F0E080935700849199819FBF0F90CF91DF910895DF93CF930F92CDB7DEB78FB76E
:206B80008983F89407B600FCFDCF89E0E2E0F0E080935700849199819FBF0F90CF91DF9177
:206BA0000895DF93CF930F92CDB7DEB78FB78983F89407B600FCFDCF89E0E1E0F0E080933A
:206BC0005700849199819FBF0F90CF91DF9108950895FC0105900020E9F7809590958E0FBF
:206BE0009F1F0895FB01DC014150504048F005900D920020C9F701C01D9241505040E0F78C
:206C00000895FB01DC0102C001900D9241505040D8F70895FB01DC0101900D920020E1F77E
:206C20000895FB01DC014150504030F08D910190801919F40020B9F7881B990B0895629F93
:206C4000D001739FF001829FE00DF11D649FE00DF11D929FF00D839FF00D749FF00D659FE5
:206C6000F00D9927729FB00DE11DF91F639FB00DE11DF91FBD01CF0111240895AA1BBB1BA3
:206C800051E107C0AA1FBB1FA617B70710F0A61BB70B881F991F5A95A9F780959095BC0175
:206CA000CD01089597FB092E07260AD077FD04D0E5DF06D000201AF4709561957F4F089523
:206CC000F6F7909581959F4F0895A1E21A2EAA1BBB1BFD010DC0AA1FBB1FEE1FFF1FA21749
:206CE000B307E407F50720F0A21BB30BE40BF50B661F771F881F991F1A9469F760957095F7
:206D0000809590959B01AC01BD01CF01089597FB092E05260ED057FD04D0D7DF0AD0001C1F
:206D200038F450954095309521953F4F4F4F5F4F0895F6F790958095709561957F4F8F4FAD
:206D40009F4F0895911106C080538A5010F0865C06C0089599278827089585FDFBCF806214
:206D60009111F8CF81568A51E0F708959111089581568A5108F4805285580895F894FFCFF1
:206D800004005730305400454E41424C45004155544F002A2E50434D004552524F52002A18
:206DA0002E2A0044495341424C45005553522041434B004D414E55414C0043414E43454C3A
:206DC000454400574149542031323820424C0001FF01525820454E41424C45204641494CDE
:206DE0004544005041434B4554204552524F52004E4F204E4554004552524F520057414999
:206E00005420464F52204D31323834204150502050524F470057524954494E47204D31328E
:206E2000383420464143544F52592044454641554C54204657005741495420464F52204D23
:206E4000313238342052455620524551004A4F494E494E47204E4554574F524B005258202C
:206E6000465720494D4700444F4E450057522031323820494D47004657205752204F4B00D1
:206E80005752203132382046570053454E44494E47004E4F5420524553504F4E44494E47BF
:206EA0000053454E54004F5441204552524F520053454E542057495448204552524F525377
:206EC000004D33323930004D31323834004D333239304644004D31323834464400454E5449
:206EE000455220544F205245434549564520465720494D41474500FFFFEF01EF0123454E41
:206F000041424C450044495341424C45004155544F004D414E55414C002A2E2A00454D500E
:206F20005459004552524F52005741495400444F4E45002A2E50434D004C4F57204241549E
:206F400054004C454156494E47204E4554574F524B004A4F494E494E47204E4554574F5280
:206F60004B00FFFF610700001A00010200000061070100030001010000001C000000EC00CD
:046F8000010001000B
:207000000C9432000C944F000C944F000C944F000C94E0010C944F000C944F000C944F0083
:207020000C944F000C944F000C944F000C944F000C944F000C944F000C944F000C944F00D8
:207040000C944F000C944F000C944F000C944F000C944F000C944F000C944F000C944F00B8
:207060000C944F0011241FBECFEFD8E0DEBFCDBF12E0A0E0B1E0E0E7FAE002C005900D92D6
:20708000A230B107D9F712E0A2E0B2E001C01D92A730B107E1F70E9451000C9436050C944B
:2070A0000000AF92BF92CF92DF92EF92FF920F931F93DF93CF9300D00F92CDB7DEB7809197
:2070C000FEFF9091FFFF9B838A83A895809160008061877F80936000809360008FEF80935D
:2070E0007E0083E080937F008FE18093640080B7806880BF83B7817F83BF8FB78983F8947E
:2071000080E88093610081E08093610089818FBFB090660080916400877F8093640010922C
:20712000700010926F008091B60088608093B6008091B60090E087709070892BC9F780E84C
:20714000D82ECC24C394AA24AA941092B2001092850010928400C092B000C0928100A7BAFF
:20716000B89BFECF1092B00010928100609184007091850080E090E00E947D027B018C0185
:2071800020E83BEE42EF56E40E944D02882324F4809166008F5F0FC020E83CE545EF56E4D4
:2071A000C801B7010E941D02181614F081E006C08091660081508093660080E0DA9419F09C
:2071C000882319F204C0882311F4B09266008091B600877F8093B6008091640088608093D7
:2071E00064001092B000109270000E94D701892B09F0FFCF8091B60088608093B600809149
:20720000B000887F8093B0008091B00081608093B00080E00E94AB01F894109264001092AD
:207220007E0010927F0095B79C7F85B7816085BF95BFE0E0F0E0099580E090E00F900F9057
:207240000F90CF91DF911F910F91FF90EF90DF90CF90BF90AF900895FF920F931F939C01E6
:2072600068EE73E00E94EB04082FF92EC90168EE73E00E94EB04FB0124E0EE0FFF1F2A9598
:20728000E1F7802F9F2D64E670E00E94EB04482F192F802F9F2D64E670E00E94EB049B016F
:2072A0002E0F3F1F94E0220F331F9A95E1F7842F912F6AE070E00E94EB04260F371F84E0A8
:2072C000220F331F8A95E1F7842F912F6AE070E00E94EB04282B392BC9011F910F91FF9036
:2072E0000895FC01EF70F070AC01452F552742954F7028EE33E0429FB001439F700D529FF7
:20730000700D11246E0F7F1F9C01207F3070A4E036952795AA95E1F7A901F3E0440F551F5E
:20732000FA95E1F7220F331F420F531F640F751F80709F70892F992724E630E0AC01429F7A
:20734000C001439F900D529F900D1124680F791FCB0108950895882319F0833039F510C0B0
:207360008091B00088678093B0008091700082608093700080EA8093B30010920202089541
:207380008091B00088678093B0008091700082608093700080EA8093B30088E090E0909369
:2073A00006028093050281E08093020208952F9A279A2F9A81E00E94AB0180E090E0089527
:2073C0001F920F920FB60F9211242F933F938F939F9380910202882339F1809103029091B7
:2073E0000402019790930402809303020196E1F48091000190E021E030E082279327809339
:207400000001882321F48091B0008F7C03C08091B00080638093B000809105029091060274
:2074200090930402809303029F918F913F912F910F900FBE0F901F901895A8E1B0E0E3E2E6
:20744000F2E00C940B0569837A838B839C832D833E834F83588789E0E82EF12CEC0EFD1EC1
:20746000B701CE0101960E941A048E010F5E1F4FB801CE0105960E941A048985823040F0F1
:207480008989823028F0B801C7010E94920401C08FEF6896E6E00C942705A8E1B0E0E3E5A7
:2074A000F2E00C940B0569837A838B839C832D833E834F83588789E0E82EF12CEC0EFD1E61
:2074C000B701CE0101960E941A048E010F5E1F4FB801CE0105960E941A048985823040F091
:2074E0008989823028F0B801C7010E94920401C081E06896E6E00C942705A8E0B0E0E3E862
:20750000F2E00C9409057B018C01611571058105910519F482E0898360C083E089838EE161
:20752000C82ED12CDC82CB82ED82FE820F831887C801B7010E94F602BC016150704077FFDE
:2075400039C0EE27FF27E61BF70B20E030E040E050E081E090E0A0E0B0E00E2E04C0880F1C
:20756000991FAA1FBB1F0A94D2F70197A109B1098E219F21A023B1230097A105B10521F043
:2075800021E030E040E050E004C016950795F794E794EA95D2F72E293F29402B512B2D83DB
:2075A0003E834F8358878EE190E0861B970B9C838B8313C06115710581F0062E04C0EE0CE8
:2075C000FF1C001F111F0A94D2F7ED82FE820F831887C61AD70ADC82CB821A82CE0101964C
:2075E0000E9445032896E8E00C942505EF92FF920F931F937B018C0180E0E81680E0F80626
:2076000081E0080780E0180788F48FEFE816F1040105110531F028F088E090E0A0E0B0E051
:2076200017C080E090E0A0E0B0E012C080E0E81680E0F80680E0080781E0180728F088E195
:2076400090E0A0E0B0E004C080E190E0A0E0B0E020E230E040E050E0281B390B4A0B5B0B61
:2076600004C016950795F794E7948A95D2F7F701EF5FFE4F8081281B310941095109C90192
:207680001F910F91FF90EF900895DF92EF92FF920F931F93FC01E480F58006811781D180D2
:2076A0008081823048F480E090E0A0E1B0E0E82AF92A0A2B1B2BA5C0843009F49FC0823023
:2076C00021F4EE24FF24870105C0E114F1040105110519F4E0E0F0E096C0628173819FEFB5
:2076E000623879070CF05BC022E83FEF261B370B2A3131052CF020E030E040E050E02AC0A7
:20770000B801A701022E04C076956795579547950A94D2F781E090E0A0E0B0E004C0880FA2
:20772000991FAA1FBB1F2A95D2F70197A109B1098E219F21A023B1230097A105B10521F060
:2077400081E090E0A0E0B0E09A01AB01282B392B4A2B5B2BDA01C9018F779070A070B07074
:2077600080349105A105B10539F427FF09C0205C3F4F4F4F5F4F04C0215C3F4F4F4F5F4FD6
:20778000E0E0F0E02030A0E03A07A0E04A07A0E45A0710F0E1E0F0E079018A0127C060387D
:2077A000710564F5FB01E158FF4FD801C7018F779070A070B07080349105A105B10539F4CD
:2077C000E7FE0DC080E490E0A0E0B0E004C08FE390E0A0E0B0E0E80EF91E0A1F1B1F17FFD7
:2077E00005C016950795F794E794319687E016950795F794E7948A95D1F705C0EE24FF241B
:207800008701EFEFF0E06E2F679566276795902F9F77D794DD24D7948E2F8695492F462BA3
:20782000582F5D29B701CA011F910F91FF90EF90DF900895FC01DB01408151812281622FAE
:207840006F7770E0221F2227221F9381892F880F822B282F30E0991F9927991F11969C93AA
:20786000119721153105A9F5411551056105710511F482E037C082E89FEF13969C938E937F
:2078800012979A01AB0167E0220F331F441F551F6A95D1F783E08C930DC0220F331F441F5B
:2078A000551F12968D919C911397019713969C938E931297203080E0380780E0480780E47B
:2078C000580758F314962D933D934D935C93179708952F3F310579F4411551056105710511
:2078E00019F484E08C93089564FF03C081E08C9312C01C9210C02F57304013963C932E9336
:20790000129783E08C9387E0440F551F661F771F8A95D1F7706414964D935D936D937C93AF
:20792000179708951F93DC01FB019C91923008F447C08081823008F443C0943051F411961D
:207940001C91843099F58181682F70E0611B71093FC0843021F0923031F48230B9F1818150
:20796000882389F12DC011961C9111978230F1F081811817D9F412962D913C911397828188
:2079800093818217930794F028173907BCF014968D919D910D90BC91A02D24813581468122
:2079A0005781281739074A075B0718F4112341F00AC082179307A407B50740F4112319F077
:2079C00061E070E005C06FEF7FEF02C060E070E0CB011F910895AA1BBB1B51E107C0AA1FBD
:2079E000BB1FA617B70710F0A61BB70B881F991F5A95A9F780959095BC01CD0108952F929E
:207A00003F924F925F926F927F928F929F92AF92BF92CF92DF92EF92FF920F931F93CF9333
:207A2000DF93CDB7DEB7CA1BDB0B0FB6F894DEBF0FBECDBF09942A88398848885F846E84F4
:207A40007D848C849B84AA84B984C884DF80EE80FD800C811B81AA81B981CE0FD11D0FB6D7
:207A6000F894DEBF0FBECDBFED010895F894FFCF0100010202030303030404040404040471
:207A8000040505050505050505050505050505050506060606060606060606060606060638
:207AA0000606060606060606060606060606060606070707070707070707070707070707F7
:207AC0000707070707070707070707070707070707070707070707070707070707070707C6
:207AE000070707070707070707070707070707070708080808080808080808080808080897
:207B0000080808080808080808080808080808080808080808080808080808080808080865
:207B2000080808080808080808080808080808080808080808080808080808080808080845
:207B4000080808080808080808080808080808080808080808080808080808080808080825
:127B60000808080808080808080808080808080808008B
:0400000500000000F7
:00000001FF
